:020000040800F2
:10000000480B002049010008AD150008A91500089B
:1000100000000000000000000000000000000000E0
:10002000000000000000000000000000311800087F
:10003000ED0400080000000029160008331800082D
:100040005D0100085D0100085D0100085D01000818
:100050005D0100085D0100085D0100085D01000808
:100060005D0100085D0100085D0100085D010008F8
:100070005D0100085D010008000000005D0100084E
:10008000000000005D01000800000000000000000A
:100090005D010008000000005D0100085D0100082E
:1000A0005D0100085D0100085D0100085D010008B8
:1000B0005D0100085D0100085D0100085D010008A8
:1000C00000F002F800F030F80CA030C8083824180E
:1000D0002D18A246671EAB4654465D46AC4201D180
:1000E00000F022F87E460F3E0FCCB6460126334282
:1000F00000D0FB1AA246AB4633431847D05100004C
:10010000F05100000023002400250026103A01D3FE
:1001100078C1FBD8520700D330C100D50B607047BF
:100120001FB51FBD10B510BD00F0DCF81146FFF77C
:10013000F7FF01F08FFD00F0F4F803B4FFF7F2FFD2
:1001400003BC00F0FBF8000008488047084800475F
:10015000FEE7FEE7FEE7FEE7FEE7FEE7FEE700005C
:1001600004480549054A064B70470000AD180008D1
:10017000C100000848050020480B00204807002067
:1001800048070020002203098B422CD3030A8B422C
:1001900011D300239C464EE003460B433CD400227F
:1001A00043088B4231D303098B421CD3030A8B4291
:1001B00001D394463FE0C3098B4201D3CB01C01A5F
:1001C000524183098B4201D38B01C01A524143092A
:1001D0008B4201D34B01C01A524103098B4201D318
:1001E0000B01C01A5241C3088B4201D3CB00C01A85
:1001F000524183088B4201D38B00C01A52414308FD
:100200008B4201D34B00C01A5241411A00D2014621
:100210005241104670475DE0CA0F00D049420310BA
:1002200000D34042534000229C4603098B422DD309
:10023000030A8B4212D3FC22890112BA030A8B42B1
:100240000CD3890192118B4208D3890192118B4200
:1002500004D389013AD0921100E08909C3098B4285
:1002600001D3CB01C01A524183098B4201D38B01C8
:10027000C01A524143098B4201D34B01C01A52416B
:1002800003098B4201D30B01C01A5241C3088B42B0
:1002900001D3CB00C01A524183088B4201D38B009B
:1002A000C01A5241D9D243088B4201D34B00C01A25
:1002B0005241411A00D20146634652415B1010463A
:1002C00001D34042002B00D54942704763465B1082
:1002D00000D3404201B50020C046C04602BD704771
:1002E00070477047754600F025F8AE460500694630
:1002F0005346C008C000854618B020B5FFF730FF50
:1003000060BC00274908B6460026C0C5C0C5C0C5A8
:10031000C0C5C0C5C0C5C0C5C0C5403D49008D46AB
:10032000704710B50446C046C0462046FFF705FF9B
:1003300010BD000000487047E40400200149182067
:10034000ABBEFEE726000200704770B58C1805783A
:10035000401C6B075B0F01D10378401C2A1106D1AA
:100360000278401C03E00678401C0E70491C5B1E9E
:10037000F9D12B0705D40023521E0DD40B70491C54
:10038000FAE70378401CCB1A921C03E01D780D702D
:10039000491C5B1C521EF9D5A142D8D3002070BD68
:1003A00070B5044600250A4800681123AB220021DD
:1003B00086680846B04700BF05E0E0B2044A12680C
:1003C000516888476D1C03488542F6D370BD000014
:1003D0006C040020180C0000FFB581B005461446DF
:1003E0002646E017800F8019811002980818401ED9
:1003F00083B204982818401E82B2134800688768A8
:1004000028460299B84710480068C069002809D0FA
:100410000A9800900C480068C66922462846049B4A
:100420000299B04700F01AF880B2009000F00EF880
:1004300086B2054800688768324600210846009B5E
:10044000B84705B0F0BD00006C04002010B50249AB
:1004500009684869804710BD6C04002010B5024946
:1004600009688869804710BD6C04002010B501241C
:100470000848094908600948094908600968086886
:100480008047FF20FFF78CFF064800F029F8002482
:10049000204610BD50040020680400207004002095
:1004A0006C0400205804002010B50B490968C86886
:1004B000804700BFFF2101310520000700F0CCF983
:1004C0000028F7D101220421044800F0CEF90A20C7
:1004D00000F00DF810BD00006C0400200004005076
:1004E000014908607047000068040020704710B59B
:1004F0000446204600F0ACF810BD000000B585B001
:100500003548C06A012108433349C8620846C06AB9
:10051000022108433049C8620846C06A02210843E4
:100520002D49C8620846C06A012108432A49C862A9
:100530000846C06A022108432749C8620120C00357
:100540000090012001900020029003200390694652
:100550000520000700F08AF80120C00200906946DB
:100560001E4800F083F80420009069461B4800F004
:100570007DF80120800200906946184800F076F866
:10058000FF20013000900020019002200290694677
:100590000520000700F06AF80022012189020F48B7
:1005A00000F063F900220121C9030520000700F0D3
:1005B0005CF90122D1030520000700F056F9012261
:1005C0000421064800F051F90A20FFF790FF01F0DE
:1005D000C3F805B000BD0000001002400004005048
:1005E00010B5044600220121C9030520000700F0D0
:1005F0003CF90122D102064800F037F9E0B201F0DF
:1006000005F90122D1030520000700F02EF910BDE5
:100610000004005010B5044600220121C903052042
:10062000000700F022F900220121C902064800F06B
:100630001CF9204601F0EAF80122D1030520000749
:1006400000F013F910BD00000004005000BFFEE7E9
:1006500031B5002400F010F9044600BF00F00CF999
:10066000001B00998842F9D338BD0000F0B503465D
:100670000A460027002400200021DAE001258D40F1
:100680002F4615683D402C46BC4276D15568022D58
:1006900002D05568122D15D1CD08AD001E4620366A
:1006A00070594D07EE0E0F25B5400646AE43304655
:1006B0004E07F60E1569B5402843CD08AE001D461D
:1006C0002035A8515568012D08D05568022D05D058
:1006D0005568112D02D05568122D18D198684E001A
:1006E0000325B5400646AE4330464E00D568B540BA
:1006F00028439860586801258D400646AE43304631
:100700001026556835402D098D40284358601868DB
:100710004E000325B5400646AE4330461579AD0779
:10072000AD0F4E00B54028431860D8684E00032531
:10073000B5400646AE4330464E009568B540284366
:10074000D8600126360755683540B54270D13B4D1B
:100750006D6B01263543394E7563394D8E08B600F1
:10076000A8598D072E0F0F25ED43B54028400525CC
:100770002D07AB4202D1002515E059E0314DAB42C7
:1007800001D101250FE0304DAB4201D102250AE035
:100790002E4DAB4201D1032505E02D4DAB4201D1D9
:1007A000042500E005258E07360FB5402843244D6B
:1007B0008E08B600A851274D28680546A54328464F
:1007C0000126360455683540B54202D10546254319
:1007D0002846204D286068680546A543284601261E
:1007E000760455683540B54202D105462543284672
:1007F000184D6860A8680546A543284601263605B9
:1008000055683540B54202D1054625432846114D6D
:10081000A860E8680546A543284601267605556880
:100820003540B54202D1054625432846094DE860CA
:10083000491C102900D221E7F0BD00000010024041
:10084000080001400004005000080050000C005057
:10085000001C005000040140024613690B40002BAD
:1008600001D0012000E000207047002A01D0816102
:1008700000E0816270470000014800687047000096
:100880000804002002480068401C014908607047C5
:100890000804002010B509480068402108430749B2
:1008A00008600846006802210843044908600320E4
:1008B00000F006F800F017F8002010BD00200240FC
:1008C00070B5044600F096F906467D21C900FFF791
:1008D00059FC054600F04CFE00222146501E00F057
:1008E00003F8002070BD704770B504460D461646EB
:1008F0002946204600F05CFE70BD000070B504463D
:100900000E460025B8480068C007C00FB0426ED23E
:10091000B5480068400840003043B34908600846C5
:100920000068C007C00FB04201D0012070BD022195
:1009300020680840022807D1AC48C068F0218843ED
:10094000A1680843A949C8602078C007C00F0028E3
:100950004CD06068022809D1A448006801214904EC
:100960000840400C002824D10120DFE760680028FF
:1009700009D19E480068012149020840400A002828
:1009800017D10120D2E76068032809D19748006891
:10099000012149060840400E00280AD10120C5E780
:1009A00092480068042108408008002801D10120F5
:1009B000BCE78E48C06880088000616808438B49A6
:1009C000C860FFF759FF05466068022810D107E0AC
:1009D000FFF752FF401B8649884201D90320A5E753
:1009E0008248C0680C2108400828F1D1DAE035E0DF
:1009F000606803280FD107E0FFF73EFF401B7C49EA
:100A0000884201D9032091E77848C0680C2108404A
:100A10000C28F1D1C6E0606800280FD107E0FFF78D
:100A20002BFF401B7249884201D903207EE76F48A3
:100A3000C0680C2108400028F1D1B3E007E0FFF7BF
:100A40001BFF401B6A49884201D903206EE76748B3
:100A5000C0680C2108400428F1D1A3E002212068DD
:100A60000840022807D16148C068F0218843A16886
:100A700008435E49C8602078C007C00F00284CD0EA
:100A80006068022809D159480068012149040840DA
:100A9000400C002824D1012048E76068002809D1D3
:100AA00052480068012149020840400A002817D135
:100AB00001203BE76068032809D14C480068012108
:100AC00049060840400E00280AD101202EE7474879
:100AD0000068042108408008002801D1012025E792
:100AE0004248C06880088000616808433F49C86088
:100AF000FFF7C2FE0546606802280FD107E0FFF746
:100B0000BBFE401B3A49884201D903200EE7374813
:100B1000C0680C2108400828F1D134E0606803283F
:100B20000FD107E0FFF7A8FE401B3149884201D9E9
:100B30000320FBE62D48C0680C2108400C28F1D1A9
:100B400021E0606800280FD107E0FFF795FE401B09
:100B50002749884201D90320E8E62448C0680C21CF
:100B600008400028F1D10EE007E0FFF785FE401BAA
:100B70001F49884201D90320D8E61C48C0680C21CF
:100B800008400428F1D1184800684008400030436C
:100B90001549086008460068C007C00FB04201D080
:100BA0000120C3E6042120680840042808D10F482A
:100BB000C068072109028843E16808430B49C860FF
:100BC000082120680840082809D10848C068072182
:100BD000C90288432169C90008430449C860032049
:100BE000FFF76EFE0020A1E6002002400010024048
:100BF0008813000010B500F013F80649C968F02208
:100C000011400909044A515CC8400449086008467B
:100C1000006810BD001002401504002028040020C8
:100C2000F8B5002400270020009000250026294860
:100C30004068072149030840450BA80026490D5884
:100C40002448C0680C210840002806D0042806D09B
:100C500008280ED00C2838D10DE02E4637E01D486C
:100C6000006810210840002801D01C4E00E01C4EF6
:100C70002DE01C4E2BE01748C0680F218904084066
:100C800004461448C0680321890508400746A00CA3
:100C900015490C5CB80D471C0E48C06801210904B9
:100CA000084000900098002807D10D49614308468C
:100CB0003946FFF767FA064606E00A4961430846E7
:100CC0003946FFF75FFA064601E02E4600BF00BF37
:100CD0003046F8BD00100240841C000800093D00A9
:100CE0000024F40000127A000C04002070B50446C1
:100CF00000252078C007C00F002871D0FC48C068CC
:100D00000C21084008280BD0F948C06808400C287E
:100D100014D1F748C06801210904084088420DD168
:100D2000F3480068012149040840400C002857D0CE
:100D300049106068884253D0012070BDEC480068BB
:100D4000052109048843EA490860FFF795FD054637
:100D500007E0FFF791FD401BE649884201D90320D7
:100D6000EBE7E3480068012149040840400C0028F3
:100D7000EFD1DF4800680521090488436168084312
:100D8000DB490860012109046068884214D1FFF73B
:100D900073FD054607E0FFF76FFD401BD54988420C
:100DA00001D90320C9E7D24800680121490408405D
:100DB000400C0028EFD013E0FFF75EFD054607E08A
:100DC000FFF75AFD401BCB49884201D90320B4E705
:100DD000C7480068012149040840400C0028EFD1B1
:100DE00002212068084002286AD1C148C0680C214D
:100DF000084004280BD0BE48C06808400C281DD10C
:100E0000BB48C068012109040840002816D1B84831
:100E10000068042108408008002804D0E068012808
:100E200001D0012089E7B24840681F2109028843A8
:100E3000216909020843AE49486041E0E0680028A2
:100E400024D0AB48006809218843E1680843A849D9
:100E50000860FFF711FD054606E0FFF70DFD401B9A
:100E6000642801D9032068E7A148006804210840EC
:100E700080080028F1D09E4840681F21090288435D
:100E80002169090208439A49486019E098480068B6
:100E900009218843E168084395490860FFF7ECFCA5
:100EA000054606E0FFF7E8FC401B642801D9032053
:100EB00043E78F4800680421084080080028F1D1EA
:100EC00010212068084010286FD18948C0680C2183
:100ED000084000281FD186480068012149020840C7
:100EE000400A002804D0E069012801D0012024E74D
:100EF0007F484068072149038843616A08437C4969
:100F00004860084640680002000A218C0906084330
:100F10007749486049E0E06900282CD074480068AF
:100F2000FF210131084372490860FFF7A5FC05461F
:100F300006E0FFF7A1FC401B642801D90320FCE672
:100F40006B480068012149020840400A0028F0D09F
:100F500067484068072149038843616A0843644938
:100F60004860084640680002000A218C09060843D0
:100F70005F49486019E05E480068FF2101318843FD
:100F80005B490860FFF778FC054606E0FFF774FC54
:100F9000401B642801D90320CFE655480068012191
:100FA00049020840400A0028F0D108212068084082
:100FB000082839D1606900281BD04D4840300069AD
:100FC000012108434A4940310861FFF755FC0546B5
:100FD00006E0FFF751FC401B642801D90320ACE672
:100FE0004348403000690221084040080028F0D002
:100FF0001AE03F4840300069400840003C49403119
:101000000861FFF739FC054606E0FFF735FC401B99
:10101000642801D9032090E6354840300069022158
:10102000084040080028F0D12021206808402028EE
:1010300049D1A069002826D000BF2D488068012131
:1010400008432B4988600846406B01210843284922
:1010500048632948006A491408432749086200BFC9
:10106000FFF70AFC054606E0FFF706FC401B642874
:1010700001D9032061E61E4880680221084040082B
:101080000028F1D01FE000BF1948806840084000E8
:10109000174988601848006A1849084016490862CC
:1010A00000BFFFF7E9FB054606E0FFF7E5FB401B45
:1010B000642801D9032040E60D48806802210840D9
:1010C00040080028F1D1042120680840042878D184
:1010D0000748806B8906084305498863084800680B
:1010E0008915084306490860FFF7C6FB054610E06E
:1010F000001002408813000000000140FEDFFFFFE7
:1011000000700040FFF7B8FB401B642801D90320A2
:1011100013E668480068FF21013108400028F1D03B
:101120006548006905210902884363490861FFF7A2
:10113000A3FB054607E0FFF79FFB401B5F49884282
:1011400001D90320F9E55C48006901214902084002
:10115000400A0028EFD15848006905210902884358
:10116000A1680843544908618915A068884214D1D0
:10117000FFF782FB054607E0FFF77EFB401B4F4968
:10118000884201D90320D8E54B4800690121490272
:101190000840400A0028EFD013E0FFF76DFB05463A
:1011A00007E0FFF769FB401B4449884201D903204F
:1011B000C3E541480069012149020840400A00286E
:1011C000EFD1A06A002872D03B484038C0680C219B
:1011D00008400C2869D0A06A022848D13648403817
:1011E0000068012109068843334940390860FFF748
:1011F00043FB054606E0FFF73FFB401B642801D98F
:1012000003209AE52C48403800680121490608402F
:10121000400E0028EFD1616B206B0843E16A084360
:1012200025494039C968FD221204914308432249E7
:101230004039C860084600680121090608431E4974
:1012400040390860FFF718FB054606E0FFF714FB7E
:10125000401B642801D903206FE517484038006817
:10126000012149060840400E0028EFD01FE0124837
:10127000403800680121090688430F494039086059
:10128000FFF7FAFA054606E0FFF7F6FA401B642876
:1012900001D9032051E5084840380068012149067A
:1012A0000840400E0028EFD101E0012045E5002074
:1012B00043E5000000700040401002408813000029
:1012C00010B50446002C01D1012010BD022151208F
:1012D0000155206800684021884321680860204645
:1012E00000F054F80021522001555120015500BF53
:1012F0005020015500BF0020E7E701465120405C27
:10130000704710B50446002C01D1012010BD5120BA
:10131000005D002802D1204600F039F8022151205A
:101320000155206800684021884321680860A16851
:1013300060680843E168084321690843616908431C
:1013400001225202A16911400843E1690843216A60
:101350000843A16A084321680860A069000C0421C1
:101360000840616A0843216848602168E06A0861B2
:101370002068C069910088432168C861002152201B
:1013800001550121512001550020BFE770477047EA
:10139000F8B504460E4615461F465120005D01284B
:1013A0007CD1002E01D0002D01D10120F8BD00BF5D
:1013B0005020005D012801D10220F7E701215020D3
:1013C000015500BF12215120015500215220015525
:1013D0002663A586E5860020E064A064A087E087F8
:1013E00001214903A06A88420DD100BF206800682E
:1013F0008843216808602068006801214903084388
:101400002168086000BF0121C903A068884205D196
:101410002068006849100843216808602068006857
:1014200040210840402804D0206800680843216813
:101430000860E068002832D16068002802D0E08EA1
:10144000012808D1216B481C206308782168C860F6
:10145000E08E401EE08612E03B460022022120463C
:1014600000F0E3F8002801D003209FE7216B481C1F
:10147000206308782168C860E08E401EE086E08E18
:101480000028E9DC01214903A06A88423AD120689A
:101490000068491008432168086033E065E060682F
:1014A000002802D0E08E012809D1206B0088216835
:1014B000C860206B801C2063E08E401EE08613E035
:1014C0003B4600220221204600F0AFF8002801D060
:1014D00003206BE7206B00882168C860206B801CAC
:1014E0002063E08E401EE086E08E0028E8DC0121CB
:1014F0004903A06A884205D1206800684910084362
:10150000216808603B4600220221204600F08DF849
:10151000002807D05220005D2021084352210855A1
:10152000032043E73B4601228021204600F07DF85E
:10153000002807D05220005D202108435221085581
:10154000032033E7A068002805D100BF2068C068E9
:101550002068806800BF01215120015500BF002193
:101560005020015500BF002020E702201EE70000A8
:1015700070B504462546681E0949884201D90120F4
:101580000CE0681E074948610321081F00F010F8AD
:1015900000200449886107200861002070BD000018
:1015A000FFFFFF0000E000E000BFFEE77047000023
:1015B00010B5002819DA1A4A03071B0F083B9B08CD
:1015C0009B00D2588307DC0EFF23A3409A438B076E
:1015D0001B0E8407E40EA3401A43114B0407240F8B
:1015E000083CA408A4001A5118E00E4A03231B0269
:1015F000D21883089B00D2588307DC0EFF23A34038
:101600009A438B071B0E8407E40EA3401A43054B35
:10161000032424021B198408A4001A5110BD0000E1
:101620001CED00E000E100E07047FFB581B004462A
:101630000E461D460027FFF71FF9074603980028AE
:101640003FD133E0681C002830D0002D04D0FFF7D4
:1016500013F9C01BA84229D920684068E0218843BB
:10166000216848602068006840218843216808603C
:1016700001214903A06A88420DD100BF206800689B
:1016800088432168086020680068012149030843F5
:101690002168086000BF01215120015500BF0021D1
:1016A0005020015500BF032005B0F0BD20688068C0
:1016B0003040B04201D1012000E000200028C1D01C
:1016C0003DE032E0681C00282FD0002D04D0FFF749
:1016D000D3F8C01BA84228D920684068E02188437D
:1016E00021684860206800684021884321680860BC
:1016F00001214903A06A88420DD100BF206800681B
:101700008843216808602068006801214903084374
:101710002168086000BF01215120015500BF002150
:101720005020015500BF0320BEE72068806830408C
:10173000B04201D1012000E000200028C2D10020E9
:10174000B2E7000010B50348FFF7BAFD00F004F857
:1017500010BD00009004002010B51348FFF7CDFD28
:10176000002820D1114810490860FF20053048604A
:1017700000210D4881601021C1610021C16001215B
:10178000416102210161002101620121490281615F
:10179000002181620721C1620021416200F008F846
:1017A0000148FFF7AEFD10BD90040020003001405D
:1017B00010B586B004461348C06A02210843114997
:1017C000C8620820019002200290012003900320AB
:1017D00004900020059001A90B48FEF747FF202048
:1017E0000190002005900220039001A90648FEF711
:1017F0003DFF0448406B0121090308430149486348
:1018000006B010BD001002400004005031B50024A5
:1018100001231B03012269460448FFF7B9FD044672
:10182000002C01D0FFF78EFF38BD0000900400208F
:10183000704710B5FFF726F810BD000000B593B053
:101840001848806B01210907084316498863164828
:1018500000680321C902884340181349086010201A
:101860000090012007900520400309900020089077
:101870000A906846FFF73AFA002801D0FEF7E6FE24
:101880000F200E9000200F901090119012900021C8
:101890000EA8FFF733F8002801D0FEF7D7FE13B0EB
:1018A00000BD0000001002400070004015480068B4
:1018B000FF2101310843134908600846C0681249F6
:1018C00008401049C86008460068104908400D49A2
:1018D0000860084680684008400088600846006844
:1018E000012189048843074908600846C068FD2132
:1018F000090488430349C86000200861C8030449FB
:1019000088607047001002400C40FF88F6FFF6FE2A
:1019100000ED00E010B52220FEF77CFE0320FEF76C
:101920005FFE2020FEF776FE10BDFFB585B01546A0
:1019300000240026002002902420FEF76BFE28469B
:10194000E917490F0918C910C900691A4DD10027B4
:101950003EE00E98C65D002E33D0002003902CE0B0
:10196000002412E0F007C00F002806D004A8005D94
:10197000FC21084004A9085505E004A8005D0321E6
:10198000084304A908557610641C042CEAD3694660
:10199000087C8001497C090108436946897C8900EB
:1019A00008436946C97C0843C0B202900298FEF71A
:1019B00017FE0398401CC0B2039003980228CFDBA7
:1019C00005E0FF20FEF70CFEFF20FEF709FE7F1C5E
:1019D000EA17920F52199210089B5A431046D20FE1
:1019E00012185210BA42B4D8A0E0002790E00E9826
:1019F000C65DE817800F40198010401CC20F00958B
:101A0000019010184110781CFEF7BCFB00293ED055
:101A1000002E33D0002003902CE0002412E0F007C9
:101A2000C00F002806D004A8005DFC21084004A9CE
:101A3000085505E004A8005D0321084304A90855E2
:101A40007610641C042CEAD36946087C8001497C2A
:101A5000090108436946897C890008436946C97CB5
:101A60000843C0B202900298FEF7BAFD0398401CEA
:101A7000C0B2039003980228CFDB48E0002E46D185
:101A8000FF20FEF7ADFDFF20FEF7AAFD3FE0E817BF
:101A9000800F40198010401CC20F00950190101853
:101AA0004110781CFEF76EFB002930D1F02E29D0B2
:101AB000002412E0F007C00F002806D004A8005D43
:101AC000FC21084004A9085505E004A8005D032195
:101AD000084304A908557610641C042CEAD369460F
:101AE000087C8001497C090108436946897C89009A
:101AF00008436946C97C0843C0B202900298FEF7C9
:101B00006FFD04E0F02E02D1FF20FEF769FD7F1C7F
:101B1000EA17920F52199210521C089B5A43104612
:101B2000D20F12185210BA4200D960E709B0F0BDC6
:101B300012207047AC20704710B50024FEF7DEFC81
:101B40001020FEF767FD0020FEF74AFD1120FEF78A
:101B500061FD0320FEF744FD4420FEF75BFD0020FD
:101B6000FEF73EFD1120FEF73BFD4520FEF752FD3E
:101B70000020FEF735FDAB20FEF732FD4E20FEF7CC
:101B800049FD0020FEF72CFD4F20FEF743FD00200D
:101B9000FEF726FDF020FEF73DFD1F20FEF720FD9D
:101BA0002120FEF737FD0320FEF71AFD2C20FEF75B
:101BB00031FDA020FEF714FD3C20FEF72BFD642034
:101BC000FEF70EFD3220FEF725FD00BF05E00449BB
:101BD000085DFEF705FD601CC4B25A2CF7DB10BD92
:101BE0006F52000810B52220FEF714FDC420FEF746
:101BF000F7FC2020FEF70EFD10BDF8B507460C4699
:101C000015461E464420FEF705FD2046FEF7E8FC7B
:101C10003046FEF7E5FC4520FEF7FCFC3846FEF7B3
:101C2000DFFC2846FEF7DCFC4E20FEF7F3FC2046E6
:101C3000FEF7D6FC4F20FEF7EDFC3846FEF7D0FC51
:101C4000F8BD10B504462420FEF7E4FC2046FEF75C
:101C5000C7FC10BD08B5FEF71DFEFEF707FCFFF739
:101C6000EDFDFF20FEF79CFB0548AC23302203214D
:101C700000900020FEF7B0FBFEF716FC00BFFEE769
:101C80000000002000FA000000F4010000E803005A
:101C900000D0070040420F0080841E0000093D0074
:101CA000FFFFFFFFFFFFFFFFFFFFFFFFFFFFFFFF44
:101CB000FFFFFFFFFFFFFFFFFFFFFFFFFFFFFFFF34
:101CC000FFFFFFFFFFFFFFFFFFFFFFFFFFFFFFFF24
:101CD000FFFFFFFFFFFFFFFFFFFFFFFFFFFFFFFF14
:101CE000FFFFFFFFFFFFFFFFFFFFFFFFFFFFFFFF04
:101CF000FFFFFFFFFFFFFFFFFFFFFFFFFFFFFFFFF4
:101D0000F0FF0003FFF0F00003FFF0FF0003FFFF10
:101D1000FFFFFFFFFFFFFFFFFFFFFFFFFFFFFFFFD3
:101D2000FFFFFFFFFFFFFFFFFFFFFFFFFFFFFFFFC3
:101D3000FFFFFFFFFFFFFFFFFFFFFFFFFFFFFC0FA6
:101D4000FFFFFF000FFFFFFFFC0FFFFFFFFFFFFF85
:101D5000FFFFFFFFFFFFFFFC0FFFFFFF000FFFFF75
:101D6000FFFC0FFFFFFFFFFFFFFFFFFFFFFFFFFF76
:101D7000FFFFFFFFFFFFFFFFFFFFFFFFFFFFC3C3EB
:101D8000FFFFFFC3C3FFFF00000000FF00000000D3
:101D9000FFFFC3C3FFFFFFC3C3FFFF00000000FF3F
:101DA00000000000FFFFC3C3FFFFFFC3C3FFFFFF2F
:101DB000FFFFFFFFFFFFFFFFFFFFFFFFFFFFFFFF33
:101DC000FFFFFFFFFFFFFFFFFC03C0FFFFFC03005F
:101DD0003FFFFC3F0F0FFF003F0F00FF003F0F00D2
:101DE000FFFC3C3F0FFFFF003C0FFFFFC0FC0FFF5D
:101DF000FFFFFFFFFFFFFFFFFFFFFFFFFFFFFFFFF3
:101E0000FFFFFFFFFFFFFFFFFFFFF0FC0FFFFFF0F3
:101E1000F3F3FFFFFC33F3FFFFFC33F3FFFC0F3C56
:101E20000FFFF3F30FFFFFF3F30FFFFFF3F3C3FF16
:101E3000FFFC0FC3FFFFFFFFFFFFFFFFFFFFFFFFE1
:101E4000FFFFFFFFFFFFFFFFFFFFFFFFFFFFFFFFA2
:101E5000FFFFFFFFFC03FFFFFFFC00C0FFFFF0F0F0
:101E600000FFFFF0F03C3FFFF0C0FC3FFFF003FC41
:101E70003FFFFC03FC3FFFF0C0FC3FFFF0F0FC3FE6
:101E8000FFFFFFFFFFFFFFFFFFFFFFFFFFFFFFFF62
:101E9000FFFFFFFFFFFFFFFFFFFFFFFFFFFFFFFF52
:101EA000FFFFFFFFFFFFFFFFFFFFFFFC0FFFFFFF35
:101EB000000FFFFFFFFC0FFFFFFFFFFFFFFFFFFF14
:101EC000FFFFFFFFFFFFFFFFFFFFFFFFFFFFFFFF22
:101ED000FFFFFFFFFFFFFFFFFFFFFFFFFFFFFFFF12
:101EE000FFFFFFFFFFFFFFFFFFFFFFFFFFFFFFFF02
:101EF000000FFFFFC000003FFC00FFF003FC3FFFAE
:101F0000FFC3FFFFFFFFFFFFFFFFFFFFFFFFFFFF1D
:101F1000FFFFFFFFFFFFFFFFFFFFFFFFFFFFFFFFD1
:101F2000FFFFFFFFFFFFFFFFFFFFFC3FFFFFC3FCC3
:101F300000FFF003FFC000003FFFFF000FFFFFFFA7
:101F4000FFFFFFFFFFFFFFFFFFFFFFFFFFFFFFFFA1
:101F5000FFFFFFFFFFFFFFFFFFFFFFFFFFFFFFFF91
:101F6000FFFFFFFFFFFFFFFFFFFFFFFFFFFFF0FF90
:101F7000FFFFF0F0FFFFFFF003FFFFFFFC0003FF98
:101F8000FFFC0003FFFFF003FFFFFFF0F0FFFFFF88
:101F9000FFF0FFFFFFFFFFFFFFFFFFFFFFFFFFFF60
:101FA000FFFFFFFFFFFFFFFFFFFFFFFFFFFFFC3F04
:101FB000FFFFFFFC3FFFFFFFFC3FFFFFFFFC3FFF7A
:101FC000FFFC00003FFFFC00003FFFFFFC3FFFFF66
:101FD000FFFC3FFFFFFFFC3FFFFFFFFC3FFFFFFF5A
:101FE000FFFFFFFFFFFFFFFFFFFFFFFFFFFFFFFF01
:101FF000FFFFFFFFFFFFFFFFFFFFFFFFFC0FFFFFE4
:10200000FFFF003FFFFFFFF03FFFFFFFFF3FFFFF2E
:10201000FFFFFFFFFFFFFFFFFFFFFFFFFFFFFFFFD0
:10202000FFFFFFFFFFFFFFFFFFFFFFFFFFFFFFFFC0
:10203000FFFFFFFFFFFFFFFFFFFFFC3FFFFFFFFC76
:102040003FFFFFFFFC3FFFFFFFFC3FFFFFFFFC3FA9
:10205000FFFFFFFC3FFFFFFFFC3FFFFFFFFC3FFFD9
:10206000FFFFFC3FFFFFFFFFFFFFFFFFFFFFFFFF43
:10207000FFFFFFFFFFFFFFFFFFFFFFFFFFFFFFFF70
:10208000FFFFFFFFFFFFFFFFFFFFFFFFFFFFFFFF60
:10209000FFFFFFF03FFFFFFFF03FFFFFFFF03FFFBD
:1020A000FFFFFFFFFFFFFFFFFFFFFFFFFFFFFFFF40
:1020B000FFFFFFFFFFFFFFFFFFFFFFFFFFFFFFFF30
:1020C000FFFFFFFFFFFFFFFFFFFF0FFFFFFFFF000F
:1020D0003FFFFFFFF003FFFFFFFFC03FFFFFFFFCDD
:1020E00003FFFFFFFFC00FFFFFFFFC00FFFFFFFF2D
:1020F000F0FFFFFFFFFFFFFFFFFFFFFFFFFFFFFFFF
:10210000FFFFFFFFFFFFFFFFFFFFFFFFC000FFFF1D
:10211000FC00000FFFF03FFF03FFF0FFFFC3FFF0E5
:10212000FFFFC3FFF0FFFFC3FFF03FFF03FFFC0013
:10213000000FFFFFC000FFFFFFFFFFFFFFFFFFFFDC
:10214000FFFFFFFFFFFFFFFFFFFFFFFFFFFFFFFF9F
:10215000FFFFFFFFFFFFF0FFFF0FFFF0FFFF0FFF8D
:10216000F0FFFF0FFFF0000003FFF0000003FFF09F
:10217000FFFFFFFFF0FFFFFFFFF0FFFFFFFFFFFF8D
:10218000FFFFFFFFFFFFFFFFFFFFFFFFFFFFFFFF5F
:10219000FFFFFFFFFFFFFFF0FFFC3FFFF03FFC0FE3
:1021A000FFF00FFF03FFF0C3FFC3FFF0F0FFC3FF1B
:1021B000F0FC3FC3FFF0FF0F03FFF0FFC00FFFF085
:1021C000FFF03FFFFFFFFFFFFFFFFFFFFFFFFFFFEE
:1021D000FFFFFFFFFFFFFFFFFC3FFFFFFFF03FFFA1
:1021E0000FFFF0FFFF0FFFF0FFFFC3FFF0FF0FC374
:1021F000FFF0FF0FC3FFF0FF0FC3FFF03C0303FF2F
:10220000FC00000FFFFF00F03FFFFFFFFFFFFFFF9D
:10221000FFFFFFFFFFFFFFFFFFFFFFFFFFFFFFFFCE
:10222000FFFFFFFFC0FFFFFFFFC03FFFFFFFC30334
:10223000FFFFFFC3C0FFFFF0C3FC0FFFF0C3FF03AE
:10224000FFF0000003FFF0000003FFF0C3FFFFFFFB
:10225000FFFFFFFFFFFFFFFFFFFFFFFFFFFFFFFF8E
:10226000FFFFFFFFFFFFFFFFFFFC3FFFFFFFF03F10
:102270000003FFF0FF0003FFF0FFC3C3FFF0FFC345
:10228000C3FFF0FFC3C3FFF03F03C3FFFC000FC356
:10229000FFFF003FFFFFFFFFFFFFFFFFFFFFFFFF0D
:1022A000FFFFFFFFFFFFFFFFFFFFFFFFFFFFFFFF3E
:1022B000C003FFFFFC00003FFFFC3C300FFFF0FFBE
:1022C0000F0FFFF0FF0F03FFF0FF0FC3FFF03C0FF6
:1022D000C3FFFC003FC3FFFF00FFC3FFFFFFFFFF83
:1022E000FFFFFFFFFFFFFFFFFFFFFFFFFFFFFFFFFE
:1022F000FFFFFFFFFFFFFFFF03FFFFFFFF03FFFFE6
:10230000FFFFC3FFFFFFFFC3FFF03FFFC3FFF0006E
:10231000FFC3FFFFC003C3FFFFFC0003FFFFFFFC81
:1023200003FFFFFFFFFFFFFFFFFFFFFFFFFFFFFFB9
:10233000FFFFFFFFFFFFFFFFFFFFFFFF00F03FFF7B
:10234000FC00000FFFF03C0303FFF0FF0FC3FFF0A2
:10235000FF0FC3FFF0FF0FC3FFF03C0303FFFC00C0
:10236000000FFFFF00F03FFFFFFFFFFFFFFFFFFF3A
:10237000FFFFFFFFFFFFFFFFFFFFFFFFFFFFFFFF6D
:10238000FFF0FFC03FFFF0FF000FFFF0FC0F03FF67
:10239000F0FC3FC3FFF03C3FC3FFFC3C3FC3FFFCEE
:1023A000030F0FFFFF00000FFFFFF000FFFFFFFF15
:1023B000FFFFFFFFFFFFFFFFFFFFFFFFFFFFFFFF2D
:1023C000FFFFFFFFFFFFFFFFFFFFFFFFFFFFFFFF1D
:1023D000FFFFFFFFFFFFFFFFFFFFFFF03F03FFFFD8
:1023E000F03F03FFFFF03F03FFFFFFFFFFFFFFFF93
:1023F000FFFFFFFFFFFFFFFFFFFFFFFFFFFFFFFFED
:10240000FFFFFFFFFFFFFFFFFFFFFFFFFFFFFFFFDC
:10241000FFFFFFFFFFFFFFFFFFFFFFF03FFFFFFF9B
:10242000FC03FFFFFFFFC3F03FFFFFF3F03FFFFFA1
:10243000FFF03FFFFFFFFFFFFFFFFFFFFFFFFFFF7B
:10244000FFFFFFFFFFFFFFFFFFFFFFFFFFFFFFFC9F
:10245000FFFFFFFFFCFFFFFFFFF03FFFFFFFF03F2D
:10246000FFFFFFC30FFFFFFF0FC3FFFFFF0FC3FF00
:10247000FFFC3FF0FFFFFC3FF0FFFFF0FFFC3FFFE2
:10248000F0FFFC3FFFFFFFFFFFFFFFFFFFFFFFFF2E
:10249000FFFFFFFFFFC3C3FFFFFFC3C3FFFFFFC378
:1024A000C3FFFFFFC3C3FFFFFFC3C3FFFFFFC3C3E0
:1024B000FFFFFFC3C3FFFFFFC3C3FFFFFFC3C3FF94
:1024C000FFFFC3C3FFFFFFC3C3FFFFFFFFFFFFFF0C
:1024D000FFFFFFFFFFFFFFFFFFFFFFFFFFFFFFF01B
:1024E000FFFC3FFFF0FFFC3FFFFC3FF0FFFFFC3F26
:1024F000F0FFFFFF0FC3FFFFFF0FC3FFFFFFC30F7F
:10250000FFFFFFF03FFFFFFFF03FFFFFFFFCFFFF7C
:10251000FFFFFCFFFFFFFFFFFFFFFFFFFFFFFFFFCE
:10252000FFFFFFFFFFFFFFFFFFFFFFFFF03FFFFF8A
:10253000FFF00FFFF0FFFF0FFFF0F0FF0FFFF0F0D5
:102540003F0FFFFFFC3F0FFFFFFF003FFFFFFFC0FC
:10255000FFFFFFFFFFFFFFFFFFFFFFFFFFFFFFFF8B
:10256000FFFFFFFFFFFFFFFFFFFFFFFFFFFFFFFF7B
:10257000FF0000FFFFF0FFFF0FFFCFFFFFCFFFCFF8
:10258000F03FF3FFCFCFCFF3FFCFCFCFC3FFF3C0E9
:10259000003FFFFFFFFFFFFFFFFFFFFFFFFFFFFF0A
:1025A000FFFFFFFFFFFFFFFFFFFFFFFFF0FFFFFF4A
:1025B000FFF03FFFFFFFF003FF0FFFF0C03F0FFFF3
:1025C000FFC0030FFFFFC3C00FFFFFC3FC0FFFFFE0
:1025D000C3000FFFF0C003FFFFF000FFFFFFF03F5D
:1025E000FFFFFFF0FFFFFFFFFFFFFFFFFFFFFFFF0A
:1025F000FFFFFFFFFFFFFFF0FFFF0FFFF000000FE7
:10260000FFF000000FFFF0FC3F0FFFF0FC3F0FFF5B
:10261000F0FC3F0FFFF0FC0F0FFFF0F0003FFFF06A
:1026200000C0FFFFFC03FFFFFFFFFFFFFFFFFFFFF7
:10263000FFFFFFFFFFFFFFFFFFFFFFFFFFFFC003E5
:10264000FFFFFF0000FFFFFC0FF03FFFF03FFC0F1C
:10265000FFF0FFFF0FFFF0FFFF0FFFF0FFFF0FFF87
:10266000F03FFC3FFFFC0FF00FFFFF0FF00FFFFFED
:10267000FFFFFFFFFFFFFFFFFFFFFFFFFFFFF0FF79
:10268000FF0FFFF000000FFFF000000FFFF0FFFF53
:102690000FFFF0FFFF0FFFF0FFFF0FFFF0FFFF0F37
:1026A000FFF03FFC0FFFFC0FF03FFFFF0000FFFFBC
:1026B000FFC003FFFFFFFFFFFFFFFFFFFFFFFFFF65
:1026C000FFFFFFFFFFFFFFFFFFF0FFFF0FFFF00027
:1026D000000FFFF000000FFFF0FC3F0FFFF0FC3F8A
:1026E0000FFFF0F00F0FFFF0F00F0FFFF0FFFF0FE5
:1026F000FFF00FF00FFFF00FF00FFFFFFFFFFFFFE6
:10270000FFFFFFFFFFFFFFFFFFFFFFFFFFFFFFF0E8
:10271000FFFF0FFFF000000FFFF000000FFFF0FCC5
:102720003F0FFFF0FC3F0FFFF0F00F0FFFF0F00F37
:102730000FFFFFFFFF0FFFFFFFF00FFFFFFFF00F87
:10274000FFFFFFFFFFFFFFFFFFFFFFFFFFFFFFFF99
:10275000FFFFFFFFFFFFC003FFFFFC00003FFFFC88
:1027600000003FFFF0FFFF0FFFF0FFFF0FFFF0F053
:10277000FF0FFFF0F0FF0FFFF0F0FC3FFFFC00F059
:102780000FFFFC00F00FFFFFF0FFFFFFFFFFFFFF59
:10279000FFFFFFFFFFFFFFFFFFFFFFF0FFFF0FFF48
:1027A000F000000FFFF000000FFFF0FC3F0FFFFFF5
:1027B000FC3FFFFFFFFC3FFFFFF0FC3F0FFFF0007F
:1027C000000FFFF000000FFFF0FFFF0FFFFFFFFF04
:1027D000FFFFFFFFFFFFFFFFFFFFFFFFFFFFFFFF09
:1027E000FFFFFFFFFFFFF0FFFF0FFFF0FFFF0FFFF7
:1027F000F0FFFF0FFFF000000FFFF000000FFFF0F1
:10280000FFFF0FFFF0FFFF0FFFF0FFFF0FFFFFFFC6
:10281000FFFFFFFFFFFFFFFFFFFFFFFFFFFFFFFFC8
:10282000FFFFFFFFFFFFFFFC00FFFFFFFC00FFFFBC
:10283000FFF0FFFFFFFFF0FFFFFFFFF0FFFF0FFFC5
:10284000F0FFFF0FFFF03FFF0FFFFC00000FFFFF47
:1028500000000FFFFFFFFF0FFFFFFFFF0FFFFFFF56
:10286000FFFFFFFFFFFFFFFFFFFFFFFFFFF0FFFF87
:102870000FFFF000000FFFF000000FFFF0FC3F0F14
:10288000FFF0FF0F0FFFFFFC03FFFFFFC0F00FFF84
:10289000FC03FC0FFFF03FFC0FFFF0FFFF0FFFF00A
:1028A000FFFF0FFFFFFFFFFFFFFFFFFFFFFFFFFF28
:1028B000FFFFFFF0FFFF0FFFF0FFFF0FFFF0000033
:1028C0000FFFF000000FFFF0FFFF0FFFF0FFFF0F03
:1028D000FFF0FFFFFFFFF0FFFFFFFFF003FFFFFF31
:1028E000F003FFFFFFFFFFFFFFFFFFFFFFFFFFFF03
:1028F000FFFFFFFFF0FFFF0FFFF000000FFFF000F2
:10290000000FFFF0FFF00FFFF0FC03FFFFFFC03FE1
:10291000FFFFFFC03FFFFFF0FC03FFFFF0FFF00FE2
:10292000FFF000000FFFF000000FFFF0FFFF0FFFB0
:10293000FFFFFFFFFFFFFFFFFFFFFFFFFFFFFFF0B6
:10294000FFFF0FFFF000000FFFF000000FFFF0FF90
:10295000C03FFFF0FC03FFFFFFC03F0FFFFC03FF82
:102960000FFFF000000FFFF000000FFFFFFFFF0F51
:10297000FFFFFFFFFFFFFFFFFFFFFFFFFFFFFFFF67
:10298000FFFFFFFFFFFFC003FFFFFF0000FFFFFC93
:102990000FF03FFFF03FFC0FFFF0FFFF0FFFF0FFD6
:1029A000FF0FFFF03FFC0FFFFC0FF03FFFFF0000A9
:1029B000FFFFFFC003FFFFFFFFFFFFFFFFFFFFFF62
:1029C000FFFFFFFFFFFFFFFFFFFFFFF0FFFF0FFF16
:1029D000F000000FFFF000000FFFF0F0FF0FFFF01E
:1029E000F0FF0FFFF0F0FF0FFFFFF0FF0FFFFFF012
:1029F0003C0FFFFFFC003FFFFFFF00FFFFFFFFFF5B
:102A0000FFFFFFFFFFFFFFFFFFFFFFFFFFFFFFFFD6
:102A1000FFFFC003FFFFFF0000FFFC3C0FF03FFC87
:102A2000003FFC0FFF00FFFF0FFF00FFFF0FFC0048
:102A30003FFC0FFC3C0FF03FFC0F0000FFFF0FC0FE
:102A400003FFFFFFFFFFFFFFFFFFFFFFFFFFFFFF92
:102A5000FFFFFFFFFFFFFFF0FFFF0FFFF000000F82
:102A6000FFF000000FFFF0FC3F0FFFF0FC3F0FFFF7
:102A7000FFFC3F0FFFFFF03F0FFFFF000C0FFFFCBD
:102A800003003FFFF0FFC0FFFFF0FFFFFFFFFFFF6E
:102A9000FFFFFFFFFFFFFFFFFFFFFFFFFFF00FC084
:102AA000FFFFF00F003FFFFC3F0C0FFFF0FC3F0F5C
:102AB000FFF0FC3F0FFFF0FC3F0FFFF0FC3F0FFF6C
:102AC000F030FC3FFFFC00F00FFFFF03F00FFFFFB3
:102AD000FFFFFFFFFFFFFFFFFFFFFFFFFFFFFFFF06
:102AE000FFFFFFFFFFC00FFFFFFFC00FFFF0FFFF63
:102AF0000FFFF0FFFF0FFFF000000FFFF000000FCF
:102B0000FFF0FFFF0FFFF0FFFF0FFFFFFFC00FFF02
:102B1000FFFFC00FFFFFFFFFFFFFFFFFFFFFFFFFF4
:102B2000FFFFFFFFFFFFFFFFFFFFFFFF0FFFFF00A4
:102B3000000FFFFC00000FFFF03FFF0FFFF0FFFF53
:102B4000FFFFF0FFFFFFFFF03FFF0FFFFC00000F54
:102B5000FFFF00000FFFFFFFFF0FFFFFFFFFFFFF63
:102B6000FFFFFFFFFFFFFFFFFFFFFFFFFF0FFFFF65
:102B7000FFF00FFFFFFF000FFFFFC00F0FFFF00080
:102B8000FFFFFFF03FFFFFFFF000FFFFFFFFC00F61
:102B90000FFFFFFF000FFFFFFFF00FFFFFFFFF0F13
:102BA000FFFFFFFFFFFFFFFFFFFFFFFFFFFFFFFF35
:102BB000FFFFFF0FFFFFFC000FFFF000000FFFF013
:102BC0000FFF0FFFFC00FF0FFFFFF003FFFFFFFFF2
:102BD00003FFFFFFF003FFFFFC00FF0FFFF00FFFFD
:102BE0000FFFF000000FFFFFFC000FFFFFFFFF0FC4
:102BF000FFFFFFFFFFFFF0FFFF0FFFF03FFC0FFFA6
:102C0000F00FF00FFFF0C3C30FFFFFF00FFFFFFF48
:102C1000FC3FFFFFFFF00FFFFFF0C3C30FFFF00FFC
:102C2000F00FFFF03FFC0FFFF0FFFF0FFFFFFFFF74
:102C3000FFFFFFFFFFFFFFFFFFFFFFFFFFFFFFFFA4
:102C4000FFFFFFFF0FFFFFFFFC0FFFF0FFF00FFF85
:102C5000F0FF030FFFF0000FFFFFF0000FFFFFF08A
:102C6000FF030FFFF0FFF00FFFFFFFFC0FFFFFFF61
:102C7000FF0FFFFFFFFFFFFFFFFFFFFFFFFFFFFF54
:102C8000FFFFFFFFFFFFFFFFFFFFFFFFF03FF00F22
:102C9000FFF00FF00FFFF0C3FF0FFFF0F03F0FFF4B
:102CA000F0FC0F0FFFF0FFC30FFFF00FF00FFFF06E
:102CB0000FFC0FFFFFFFFFFFFFFFFFFFFFFFFFFF07
:102CC000FFFFFFFFFFFFFFFFFFFFFFFFFFFFFFFF14
:102CD000FFFFFFFFFFFFFFFFFFFFFFFFFFFFFFFF04
:102CE000FC0000000FFC0000000FFC3FFFFF0FFC8A
:102CF0003FFFFF0FFFFFFFFFFFFFFFFFFFFFFFFF94
:102D0000FFFFFFFFFFFFFFFFFFFFFFFFFFFFFFFFD3
:102D1000FFFFFFFFFFFFFFFFFFFFFFF0FFFFFFFCD5
:102D200000FFFFFFC00FFFFFFC03FFFFFFC03FFFDF
:102D3000FFF003FFFFFF003FFFFFFF0FFFFFFFFF5D
:102D4000FFFFFFFFFFFFFFFFFFFFFFFFFFFFFFFF93
:102D5000FFFFFFFFFFFFFFFFFFFFFFFFFFFFFFFF83
:102D6000FFFFFC3FFFFF0FFC3FFFFF0FFC000000D9
:102D70000FFC0000000FFFFFFFFFFFFFFFFFFFFF43
:102D8000FFFFFFFFFFFFFFFFFFFFFFFFFFFFFFFF53
:102D9000FFFFFFFFFFFFFFFFFFFFFFFFFFFFFFFF43
:102DA000FFC3FFFFFFFFF0FFFFFFFFFC3FFFFFFF41
:102DB000FF0FFFFFFFFFC3FFFFFFFF0FFFFFFFFC42
:102DC0003FFFFFFFF0FFFFFFFFC3FFFFFFFFFFFF1E
:102DD000FFFFFFFFFFFFFFFFFFFF0FFFFFFFFF0FE3
:102DE000FFFFFFFF0FFFFFFFFF0FFFFFFFFF0FFFC3
:102DF000FFFFFF0FFFFFFFFF0FFFFFFFFF0FFFFFB3
:102E0000FFFF0FFFFFFFFF0FFFFFFFFF0FFFFFFFA2
:102E1000FF0FFFFFFFFF0FFFFFFFFF0FFFFFFFFF92
:102E2000FFFFFFFFFFFFFFFFFFFFFFFFFFFFFFFFB2
:102E3000FFFFFFFFFFFFFFFFFFFFFFFFFFF3FFFFAE
:102E4000FFFFCFFFFFFFFFCFFFFFFFFF3FFFFFFFB2
:102E5000FFFFFFFFFFFFFFFFFFFFFFFFFFFFFFFF82
:102E6000FFFFFFFFFFFFFFFFFFFFFFFFFFFFFFFF72
:102E7000FFFC0FFFFFFFF003CFFFFFF0C0C3FFFF1A
:102E8000F0F0C3FFFFF0F0C3FFFFFC30C3FFFFF023
:102E90000003FFFFF0000FFFFFF0FFFFFFFFFFFF4A
:102EA000FFFFFFFFFFFFFFFFFFFFFFFFFFFFFFFF32
:102EB000FFFFF0FFFFC3FFF0000003FFF00000037F
:102EC000FFFC3F0FFFFFF0FFC3FFFFF0FFC3FFFF5B
:102ED000F0FFC3FFFFF0FFC3FFFFFC3F0FFFFFFC4E
:102EE000000FFFFFFFC0FFFFFFFFFFFFFFFFFFFF20
:102EF000FFFFFFFFFFFFFFFFFFFFFFFFFFFF00FFE1
:102F0000FFFFFC000FFFFFF03F0FFFFFF0FFC3FFCD
:102F1000FFF0FFC3FFFFF0FFC3FFFFF0FFC3FFFFA2
:102F2000F0FFCFFFFFFC3C03FFFFFC3C03FFFFFF74
:102F3000FFFFFFFFFFFFFFFFFFFFFFFFFFFFFFFFA1
:102F4000FFFFFFFF00FFFFFFFC000FFFFFFC3F0F35
:102F5000FFFFF0FFC3FFFFF0FFC3FFFFF0FFC3FF62
:102F6000FFF0FFC3FFFFFC3F0FC3FFF0000003FFB4
:102F7000F0000003FFF0FFFFFFFFFFFFFFFFFFFF79
:102F8000FFFFFFFFFFFFFFFFFFFFC0FFFFFFFC0092
:102F90000FFFFFFC300FFFFFF0F0C3FFFFF0F0C3A7
:102FA000FFFFF0F0C3FFFFF0F0C3FFFFF0F00FFFF3
:102FB000FFFC300FFFFFFC30FFFFFFFFFFFFFFFFB5
:102FC000FFFFFFFFFFFFFFFFFFFFFFFFFFFFFFFF11
:102FD000FFFFFFFFF0FFC3FFFFF0FFC3FFFFF000A5
:102FE000000FFFF0000003FFF0FFC3C3FFF0FFC3BB
:102FF000C3FFF0FFC3C3FFF0FFC3C3FFFFFFFFC367
:10300000FFFFFFFFFFFFFFFFFFFFFFFFFFFFFFFFD0
:10301000FFFFFFFFFFFFC0FFFFFFFC000FFFF0FC03
:103020003F0FFFF0F0FFC3FFF0F0FFC3FFF0F0FF32
:10303000C3FFF0F0FFC3FFF03C3F0FFFFC000003B5
:10304000FFFF000003FFFFFFFFC3FFFFFFFFFFFFC6
:10305000FFFFFFFFFFFFFFFFFFFFFFF0FFFFC3FFCB
:10306000F0000003FFF0000003FFF0FF0FFFFFFF81
:10307000FFC3FFFFFFFFC3FFFFF0FFC3FFFFF00031
:1030800003FFFFF0000FFFFFF0FFFFFFFFFFFFFF59
:10309000FFFFFFFFFFFFFFFFFFFFFFFFFFFFFFFF40
:1030A000FFFFFFFFFFFFF0FFC3FFFFF0FFC3FFFFC6
:1030B000F0FFC3FFFFF00003C3FFF00003C3FFF006
:1030C000FFFFFFFFF0FFFFFFFFF0FFFFFFFFFFFF2E
:1030D000FFFFFFFFFFFFFFFFFFFFFFFFFFFFFFFF00
:1030E000FFFFFFFFFFFFFFFFFFFFFFF0FFFFFFFFFF
:1030F000F0FFFFC3FFF0FFFFC3FFF0FFFFC3FFF0D0
:10310000FFFFC3C3F0FFFFC3C3FC000003FFFF00CA
:103110000003FFFFFFFFFFFFFFFFFFFFFFFFFFFFBA
:10312000FFFFFFFFFFFFFFFFFFFFFFFFFFF0FFFFBE
:10313000C3FFF0000003FFF0000003FFFFF0FFFFFC
:10314000FFFFC003FFFFF00F03FFFFF03FC3FFFFD0
:10315000F0FFC3FFFFF0FFC3FFFFF0FFFFFFFFFF24
:10316000FFFFFFFFFFFFFFFFFFFFFFFFFFFFFFFF6F
:10317000FFFFFFFFFFFFFFFFF0FFFFC3FFF0FFFFB9
:10318000C3FFF0FFFFC3FFF0000003FFF0000003E8
:10319000FFF0FFFFFFFFF0FFFFFFFFF0FFFFFFFF6C
:1031A000FFFFFFFFFFFFFFFFFFFFFFFFFFFFFFFF2F
:1031B000FFFFFFFFF0FFC3FFFFF00003FFFFF00082
:1031C00003FFFFF0FFC3FFFFFFFFC3FFFFF000039C
:1031D000FFFFF0000FFFFFF0FFC3FFFFFFFFC3FF84
:1031E000FFF00003FFFFF0000FFFFFF0FFFFFFFF06
:1031F000FFFFFFFFFFFFFFFFFFFFFFFFFFFFFFF0EE
:10320000FFC3FFFFF00003FFFFF00003FFFFF0FF2D
:103210000FFFFFFFFFC3FFFFFFFFC3FFFFF0FFC371
:10322000FFFFF00003FFFFF0000FFFFFF0FFFFFFC5
:10323000FFFFFFFFFFFFFFFFFFFFFFFFFFFFFFFF9E
:10324000FFFFFFFFFFFFC0FFFFFFFC000FFFFFFCC2
:103250003F0FFFFFF0FFC3FFFFF0FFC3FFFFF0FFD3
:10326000C3FFFFF0FFC3FFFFFC3F0FFFFFFC000F9A
:10327000FFFFFFC0FFFFFFFFFFFFFFFFFFFFFFFF9D
:10328000FFFFFFFFFFF0FFFFC3FFF0000003FFF0B1
:10329000000003FFF0FC3F0FFFF0F0FFC3FFFFF063
:1032A000FFC3FFFFF0FFC3FFFFF0FFC3FFFFFC3FC3
:1032B0000FFFFFFC000FFFFFFFC0FFFFFFFFFFFF3F
:1032C000FFFFFFFFFFFFFFFFFFFFFFFFFFFFFFFF0E
:1032D000FFFFC0FFFFFFFC000FFFFFFC3F0FFFFFE2
:1032E000F0FFC3FFFFF0FFC3FFFFF0FFC3FFF0F0ED
:1032F000FFC3FFF0FC3F0FFFF0000003FFF00000F2
:1033000003FFF0FFFFC3FFFFFFFFFFFFFFFFFFFF14
:10331000FFFFFFFFFFFFFFF0FFC3FFFFF0FFC3FF53
:10332000FFF00003FFFFF00003FFFFF0FC3FFFFF93
:10333000F0FF0FFFFFF0FFC3FFFFF0FFC3FFFFFF32
:10334000FF03FFFFFFFF0FFFFFFFFFFFFFFFFFFF79
:10335000FFFFFFFFFFFFFFFFFFFFFFFFFFFFFFFF7D
:10336000FFFFF03C0FFFFFF0300FFFFFF0F0C3FF57
:10337000FFF0F0C3FFFFF0C3C3FFFFF0C3C3FFFFC5
:10338000FC0303FFFFFC0F03FFFFFFFFFFFFFFFF37
:10339000FFFFFFFFFFFFFFFFFFFFFFFFFFFFFFFF3D
:1033A000FFFFFFFFFFC3FFFFFFFFC3FFFFFC0000A6
:1033B0000FFFF000000FFFF0FFC3FFFFF0FFC3FFA0
:1033C000FFF0FFC3FFFFF0FFC3FFFFFC3FC3FFFFA2
:1033D000FC3FFFFFFFFFFFFFFFFFFFFFFFFFFFFFC0
:1033E000FFFFFFFFFFFFFFFFFFFFFFC3FFFFFC002B
:1033F00003FFFFF00003FFFFF0FFFFFFFFF0FFFF01
:10340000FFFFF0FFFFFFFFFC3FC3FFFFF00003FFE4
:10341000FFF00003FFFFF0FFFFFFFFFFFFFFFFFFD5
:10342000FFFFFFFFFFFFFFFFFFFFFFFFC3FFFFFFE8
:10343000FF03FFFFFFF003FFFFFF00C3FFFFF00FDD
:10344000FFFFFFF0FFFFFFFFF00FFFFFFFFF00C3D5
:10345000FFFFFFF003FFFFFFFF03FFFFFFFFC3FFBF
:10346000FFFFFFFFFFFFFFFFFFFFFFFFFFFFFFFF6C
:10347000FFFFC3FFFFFFF003FFFFF00003FFFFF0BC
:103480000FC3FFFFFF03FFFFFFFFF03FFFFFFF033F
:10349000FFFFFFF00FC3FFFFF00003FFFFFFF0038C
:1034A000FFFFFFFFC3FFFFFFFFFFFFFFFFFFFFFF68
:1034B000FFFFFFFFFFFFFFFFFFFFFFF0FFC3FFFF67
:1034C000F0FFC3FFFFF03F03FFFFF00C03FFFFFF20
:1034D000C0FFFFFFFFC0FFFFFFF00C03FFFFF03F47
:1034E00003FFFFF0FFC3FFFFF0FFC3FFFFFFFFFF7E
:1034F000FFFFFFFFFFFFFFFFFFFFFFF0FFFFC3FF27
:10350000F0FFFF03FFF0FFF003FFF03F00C3FFF009
:10351000000FFFFFF0C03FFFFFF0FC0FFFFFFFFFBA
:1035200000C3FFFFFFF003FFFFFFFF03FFFFFFFFED
:10353000C3FFFFFFFFFFFFFFFFFFFFFFFFFFFFFFD7
:10354000FFFFFFFFFFFFFFFFFFFFFFFFF0FF03FF96
:10355000FFF03F03FFFFF00FC3FFFFF0C3C3FFFF08
:10356000F0F0C3FFFFF0FC03FFFFF03F03FFFFF0AD
:103570003FC3FFFFFFFFFFFFFFFFFFFFFFFFFFFF57
:10358000FFFFFFFFFFFFFFFFFFFFFFFFFFFFFFFF4B
:10359000FFFFFFFFFFFFFFFFF3FFFFFFFFC0FFFF86
:1035A000FF0000000FFC000C0003FC3FFFFFC3FC0A
:1035B0003FFFFFC3FFFFFFFFFFFFFFFFFFFFFFFF17
:1035C000FFFFFFFFFFFFFFFFFFFFFFFFFFFFFFFF0B
:1035D000FFFFFFFFFFFFFFFFFFFFFFFFFFFFFFFFFB
:1035E000FFFFFFFFFFFFFC00000003FC00000003E3
:1035F000FFFFFFFFFFFFFFFFFFFFFFFFFFFFFFFFDB
:10360000FFFFFFFFFFFFFFFFFFFFFFFFFFFFFFFFCA
:10361000FFFFFFFFFFFFFFFFFFFFFFFFFFFC3FFF7D
:10362000FFC3FC3FFFFFC3FC000C0003FF000000D2
:103630000FFFFFC0FFFFFFFFF3FFFFFFFFFFFFFFD5
:10364000FFFFFFFFFFFFFFFFFFFFFFFFFFFFFFFF8A
:10365000FFFFFFFFFFFFFFFFFFFFFFFFFFFFFFFF7A
:10366000FC3FFFFFFFFC3FFFFFFFFF0FFFFFFFFFE0
:103670000FFFFFFFFC0FFFFFFFF03FFFFFFFF0FF1B
:10368000FFFFFFF0FFFFFFFFF03FFFFFFFFC3FFFEB
:10369000FFFFFFFFFFFFFFFFFFFFFFFFFFFFFFFF3A
:1036A000FFFFFFFFFFFFFFFFFFFFFFFFFFFFFFFF2A
:1036B000FFFFFFFFFFFFFFFFFFFFFFFFFFFFFFFF1A
:1036C000FFFFFFFFFFFFFFFFFFFFFFFFFFFFFFFF0A
:1036D000FFFFFFFFFFFFFFCC0003FFCC0003FFFF56
:1036E000FFFFFFFFFFFFFFFFFFFFFFFFFFFFFFFFEA
:1036F000FFFFFFFFFFFFFFFFFFFFFFFFFFFFFFFFDA
:10370000FF0FFFFFC00FFFFFFF0FFFFFFFFFFFFFD8
:10371000FF0FFFFFC00FFFFFFF0FFFFFFFFFFFFFC8
:10372000FFFFFFFFFFFFFFFF33FFFF0003FFFF006F
:103730000003FFFF3003FF0003FFFF000003FFFF54
:103740003003FFFF33FFFFFFFFFFFFFFFFFFFFFF20
:10375000FFFFFFC0FC0FFFC0F003FFCFC0F3FC0F63
:10376000C3F0FFCF03F3FFC00F03FFF03F03FFFFE2
:10377000FFFFFFFFFFFFFFFFFFFFFFFFFFFFFFFF59
:103780003F0FFFFF0CF3FFFFCCF3FFFFC30FFFF072
:10379000C3FFFFCF33FFFFCF30FFFFF0FCFFFFFF82
:1037A000FFFFFFFFFFFFFFFFFFFFFFF0FFFFFFC077
:1037B000303FFFCF000FFFCC0FCFFFF0FFCFFFC098
:1037C0003FCFFFCF3FCFFFFFFFFFFFFFFFFFFFFF19
:1037D000FFFFFFFFFFFFFFFFFFFFFFFFFFFFFFFFF9
:1037E000FFFFFFFFFF0FFFFFC00FFFFFFF0FFFFFF8
:1037F000FFFFFFFFFFFFFFFFFFFFFFFFFFFFFFFFD9
:10380000FFFFFFFFFFFFFFFFFFFFFFF000FFFFC015
:10381000003FFC03FC03FC3FFFC3FFFFFFFFFFFF74
:10382000FFFFFFFFFFFFFFFFFFFFFFFFFFFFFFFFA8
:10383000FFFFFC3FFFC3FC03FC03FFC0003FFFF0A2
:1038400000FFFFFFFFFFFFFFFFFFFFFFFFFFFFFF87
:10385000FFFFFFFFFFFFFFFFFFFFFFFFFC3FFFFF3B
:103860000C3FFFFF003FFFFFF003FFFFF003FFFFF0
:10387000003FFFFF0C3FFFFFFC3FFFFFFFFFFFFF8D
:10388000FFFFFFFFFFFFFFFFCFFFFFFFCFFFFFFFA8
:10389000CFFFFFF0003FFFFFCFFFFFFFCFFFFFFF96
:1038A000CFFFFFFFFFFFFFFFFFFFFFFFFFFFFFFF58
:1038B000FFFFFFFFFFFFFFFFFFFFF03FFFFFFF03E3
:1038C000FFFFFFF3FFFFFFFFFFFFFFFFFFFFFFFF14
:1038D000FFFFFFFFFFFFFFFFFFFFFFFFFFFFFFFFF8
:1038E000CFFFFFFFCFFFFFFFCFFFFFFFCFFFFFFFA8
:1038F000CFFFFFFFCFFFFFFFCFFFFFFFFFFFFFFF68
:10390000FFFFFFFFFFFFFFFFFFFFFFFFFFFFFFFFC7
:10391000FFFFFFC3FFFFFFC3FFFFFFFFFFFFFFFF2F
:10392000FFFFFFFFFFFFFFFFFFFFFFFFFFFFFFFFA7
:10393000FFFFFFFFFFFFFC3FFFFFFC03FFFFFFC098
:103940003FFFFFFC0FFFFFFFC0FFFFFFF00FFFFF78
:10395000FF00FFFFFFF0FFFFFFFFFFFFFFFFFFFF85
:10396000FFFFFFFC003FFFF0000FFFC3FFC3FFCFCF
:10397000FFF3FFC3FFC3FFF0000FFFFC003FFFFF9B
:10398000FFFFFFFFFFFFFFFFFFFFFFFFFFFFFFCF77
:10399000FFCFFFCFFFCFFFCFFFCFFFC00003FFC0A0
:1039A0000003FFCFFFFFFFCFFFFFFFCFFFFFFFFFB2
:1039B000FFFFFFFFFFFFFFFFFFFFFFC3FC3FFFC055
:1039C000FC0FFFCC3FC3FFCF0FF3FFCFC3F3FFCFFD
:1039D000F003FFCFFC0FFFFFFFFFFFFFFFFFFFFF25
:1039E000FFFFFFF3FFCFFFC3FFC3FFCFF3F3FFCF13
:1039F000F3F3FFCFF3F3FFCFC0F3FFC00003FFF0FB
:103A00000F0FFFFFFFFFFFFFFFFFFFFFFFFFFFFFA6
:103A1000FFFFFFFC3FFFFFFC03FFFFCCF03FFFCCAD
:103A2000FF03FFC00003FFC00003FFCCFFFFFFFF49
:103A3000FFFFFFFFFFFFFFFFFFFFFFFFFFFFFFF3A2
:103A4000FFFFFFCFC003FFCFF003FFCFF3F3FFCFA4
:103A5000F3F3FFC003F3FFF00FF3FFFFFFFFFFFFE0
:103A6000FFFFFFFFFFFFFFFFFFFFFFFC00FFFFF077
:103A7000003FFFC3CF0FFFCFF3C3FFCFF3F3FFC070
:103A800003F3FFF00FF3FFFFFFFFFFFFFFFFFFFF59
:103A9000FFFFFFFFFFFFFFFFFFC3FFFFFFF3FFFF7E
:103AA000FFF3FFC0FFF3FFC000F3FFFF0003FFFFC2
:103AB000FF03FFFFFFFFFFFFFFFFFFFFFFFFFFFF12
:103AC000FFFFFFF00C0FFFC00003FFCFF3F3FFCFAA
:103AD000F3F3FFCFF3F3FFC00003FFF00C0FFFFF82
:103AE000FFFFFFFFFFFFFFFFFFFFFFFFFFFFFFCF16
:103AF000F00FFFCFC003FFCFCFF3FFC3CFF3FFF033
:103B0000F3C3FFF0000FFFFF003FFFFFFFFFFFFFCA
:103B1000FFFFFFFFFFFFFFFFFFFFFFFFFFFFFFFFB5
:103B2000FFFFFFC3F0FFFFC3F0FFFFFFFFFFFFFF3B
:103B3000FFFFFFFFFFFFFFFFFFFFFFFFFFFFFFFF95
:103B4000FFFFFFFFFFFFFFFFFFFFFFFFFFFFFC3F48
:103B5000FFFFFFC3FFFFFFF3F0FFFFFFF0FFFFFFDB
:103B6000FFFFFFFFFFFFFFFFFFFFFFFFFFFFFFFF65
:103B7000CFFFFFFFCFFFFFFF33FFFFFF33FFFFFC50
:103B8000FCFFFFF3FF3FFFF3FF3FFFCFFFCFFFCF70
:103B9000FFCFFFFFFFFFFFFFFFFFFFFFFFFFFFFF65
:103BA00033FFFFFF33FFFFFF33FFFFFF33FFFFFF55
:103BB00033FFFFFF33FFFFFF33FFFFFFFFFFFFFF79
:103BC000FFFFFFFFFFFFFFCFFFCFFFCFFFCFFFF3D1
:103BD000FF3FFFF3FF3FFFFCFCFFFFFF33FFFFFF53
:103BE00033FFFFFFCFFFFFFFCFFFFFFFFFFFFFFF11
:103BF000FFFFFFFFFFFFFFFFFC3FFFFFFC0FFFCCBE
:103C00003FCFFFCC0FCFFFFFCFCFFFFFC00FFFFF96
:103C1000F03FFFFFFFFFFFFFFFFFFFFFFFFFFFFF83
:103C2000FFFFFFF0003FFFCFFFCFFF3F0FF3FF3C51
:103C3000F3F3FF3CF3F3FFCC000FFFFFFFFFFFFFA9
:103C4000FFFFFFFFFFFFFFFFFFFFFFCFFFFFFFC0F3
:103C5000FFCFFFC003CFFFCF000FFFFF3F0FFFFFDE
:103C60003F0FFFCF000FFFC003FFFFC0FFFFFFCFDD
:103C7000FFFFFFFFFFFFFFCFFFCFFFC0000FFFC021
:103C8000000FFFCFCFCFFFCFCFCFFFCFCFCFFFC022
:103C9000000FFFF0303FFFFFFFFFFFFFFFFFFFFFC1
:103CA000FFFFFFFC00FFFFF0003FFFC3FF0FFFCF50
:103CB000FFCFFFCFFFCFFFCFFFCFFFCFFFCFFFF370
:103CC000FF3FFFFCFC0FFFFFFFFFFFFFFFFFFFCFEA
:103CD000FFCFFFC0000FFFC0000FFFCFFFCFFFCF10
:103CE000FFCFFFCFFFCFFFC3FF0FFFF0003FFFFC71
:103CF00000FFFFFFFFFFFFFFFFFFFFCFFFCFFFC072
:103D0000000FFFC0000FFFCFCFCFFFCFCFCFFFCF30
:103D100003CFFFCFFFCFFFC0FC0FFFFFFFFFFFFF71
:103D2000FFFFFFFFFFFFFFCFFFCFFFC0000FFFC070
:103D3000000FFFCFCFCFFFCFCFCFFFFF03CFFFFFCE
:103D4000FFCFFFFFFC0FFFFFFFFFFFFFFFFFFFFFA6
:103D5000FFFFFFFC00FFFFF0003FFFC3FF0FFFCF9F
:103D6000FFCFFFCF3FCFFFCF3FCFFFC03F3FFFC0D1
:103D70003C0FFFFF3FFFFFFFFFFFFFFFFFFFFFCFF6
:103D8000FFCFFFC0000FFFC0000FFFCFCFCFFFFF5F
:103D9000CFFFFFCFCFCFFFC0000FFFC0000FFFCF7F
:103DA000FFCFFFFFFFFFFFFFFFFFFFFFFFFFFFCF83
:103DB000FFCFFFCFFFCFFFCFFFCFFFC0000FFFC070
:103DC000000FFFCFFFCFFFCFFFCFFFCFFFCFFFFF12
:103DD000FFFFFFFFFFFFFFF03FFFFFC03FFFFFCFF1
:103DE000FFCFFFCFFFCFFFCFFFCFFFC0000FFFF010
:103DF000000FFFFFFFCFFFFFFFCFFFFFFFFFFFFF22
:103E0000FFFFFFCFFFCFFFC0000FFFC0000FFFCFAE
:103E10000FCFFFFF03FFFFFC30CFFFC0FC0FFFC33E
:103E2000FF0FFFCFFFCFFFFFFFFFFFFFFFFFFFCF22
:103E3000FFCFFFCFFFCFFFC0000FFFC0000FFFCFAE
:103E4000FFCFFFCFFFCFFFCFFFFFFFCFFFFFFFC0B1
:103E50003FFFFFFFFFFFFFCFFFCFFFC0000FFFC0FF
:103E6000000FFFCFF0FFFFCF03FFFFFC3FFFFFCFAF
:103E700003FFFFCFF0FFFFC0000FFFC0000FFFCF19
:103E8000FFCFFFFFFFFFFFCFFFCFFFC0000FFFC03F
:103E9000000FFFCFF0FFFFFF03FFFFFC3FCFFFC08E
:103EA000000FFFC0000FFFFFFFCFFFFFFFFFFFFF6F
:103EB000FFFFFFFC00FFFFF0003FFFC3FF0FFFCF3E
:103EC000FFCFFFCFFFCFFFCFFFCFFFC3FF0FFFF02D
:103ED000003FFFFC00FFFFFFFFFFFFFFFFFFFFCFE3
:103EE000FFCFFFC0000FFFC0000FFFCF3FCFFFCFBE
:103EF0003FCFFFCF3FCFFFFF000FFFFFC03FFFFFD0
:103F0000FFFFFFFFFFFFFFFFFFFFFFFC00FFFFF0D2
:103F1000003FFCC3FF0FFC0FFFCFFC0FFFCFFCCF18
:103F2000FFCFFCC3FF0FFC30003FFF3C00FFFFFF53
:103F3000FFFFFFFFFFFFFFCFFFCFFFC0000FFFC05E
:103F4000000FFFCFCFCFFFCFCFCFFFFF0FCFFFF0BF
:103F5000300FFFC0F03FFFCFFFFFFFCFFFFFFFFF9E
:103F6000FFFFFFFFFFFFFFC0F03FFFC0C00FFFCF0D
:103F7000C3CFFFCFCFCFFFCF0FCFFFC00C0FFFF0CE
:103F80003C0FFFFFFFFFFFFFFFFFFFFFFFFFFFFFF4
:103F9000F00FFFCFFFCFFFCFFFCFFFC0000FFFC05D
:103FA000000FFFCFFFCFFFCFFFCFFFFFF00FFFFFCF
:103FB000FFFFFFFFFFFFFFFFFFFFFFFFFFCFFFF050
:103FC000000FFFF0000FFFCFFFCFFFCFFFFFFFCFAE
:103FD000FFCFFFF0000FFFF0000FFFFFFFCFFFFF4D
:103FE000FFFFFFFFFFFFFFFFFFCFFFFFFC0FFFFF04
:103FF000000FFFC003CFFFC3FFFFFFC003CFFFFFD2
:10400000000FFFFFFC0FFFFFFFCFFFFFFFFFFFFFD2
:10401000FFCFFFFFC00FFFC0000FFFC0FFCFFFF0BB
:1040200003CFFFFFC0FFFFF003CFFFC0FFCFFFC0F4
:10403000000FFFFFC00FFFFFFFCFFFFFFFFFFFCF0E
:10404000FFCFFFC3FF0FFFC0FC0FFFCC00CFFFFF70
:1040500003FFFFCC00CFFFC0FC0FFFC3FF0FFFCF5C
:10406000FFCFFFFFFFFFFFFFFFFFFFFFFFCFFFFFC0
:10407000FF0FFFCFFC0FFFCFF0CFFFC003FFFFC04C
:1040800003FFFFCFF0CFFFCFFC0FFFFFFF0FFFFFBE
:10409000FFCFFFFFFFFFFFFFFFFFFFC3FC0FFFC0CE
:1040A000FFCFFFCC3FCFFFCF03CFFFCFF0CFFFCF6E
:1040B000FC0FFFC0FF0FFFFFFFFFFFFFFFFFFFFF32
:1040C000FFFFFFFFFFFFFFFFFFFFFFFFFFFFFFFF00
:1040D000FFFFFC000003FC000003FCFFFFF3FCFFFC
:1040E000FFF3FFFFFFFFFFFFFFFFFFFFFFFFFFFFEC
:1040F000FFFFFFFFFFF0FFFFFF00FFFFF00FFFFFDD
:10410000C0FFFFFC0FFFFFC03FFFFC03FFFFFC3FB2
:10411000FFFFFFFFFFFFFFFFFFFFFFFFFFFFFFFFAF
:10412000FFFFFCFFFFF3FCFFFFF3FC000003FC00BC
:104130000003FFFFFFFFFFFFFFFFFFFFFFFFFFFF8A
:10414000FFFFFFFFFFFFFFFFFFFFFFFFF0FFFFFF8E
:10415000FF3FFFFFFFC3FFFFFFFCFFFFFFC3FFFFAA
:10416000FF3FFFFFF0FFFFFFFFFFFFFFFFFF3FFFEE
:10417000FFFF3FFFFFFF3FFFFFFF3FFFFFFF3FFF4F
:10418000FFFF3FFFFFFF3FFFFFFF3FFFFFFF3FFF3F
:10419000FFFF3FFFFFFF3FFFFFFFFFFFFFFFFFFFAF
:1041A000FFFFFFFFFFFFFFFFFFFFFFFFFFFCFFFF22
:1041B000FFF3FFFFFFCFFFFFFFFFFFFFFFFFFFFF4B
:1041C000FFFFFFFFFFFFFFFFFFFFFFFFFFFFFFF00E
:1041D000FFFFFFC03CFFFFCF3CFFFFCF3CFFFFF3E3
:1041E0003CFFFFC000FFFFC003FFFFCFFFFFFFFF4B
:1041F000FFFFFFFFFFFFFFCFFFF3FFC00003FFC084
:104200000003FFF3F3FFFFCFFCFFFFCFFCFFFFC373
:10421000F0FFFFF003FFFFFC0FFFFFFFFFFFFFFFBB
:10422000FFFFFFFC0FFFFFF003FFFFC3F0FFFFCF17
:10423000FCFFFFCFFCFFFFCFFCFFFFC3F3FFFFF04E
:10424000C0FFFFFFFFFFFFFFFFFFFFFFFFFFFFFCC0
:104250000FFFFFF003FFFFC3F0FFFFCFFCFFFFCF17
:10426000FCFFFFF3F3F3FFC00003FFC00003FFCF29
:10427000FFFFFFFFFFFFFFFFFFFFFFFC0FFFFFF050
:1042800003FFFFC330FFFFCF3CFFFFCF3CFFFFCF5B
:1042900030FFFFC303FFFFF30FFFFFFFFFFFFFFF31
:1042A000FFFFFFFFFFFFFFFFFFFFFFCFFCFFFFCF81
:1042B000FCFFFFC0000FFFC00003FFCFFCF3FFCFE8
:1042C000FCF3FFCFFCF3FFFFFFF3FFFFFFF3FFFF64
:1042D000FFFFFFFC0FFFFFF003FFF3C3F0FFF3CF7F
:1042E000FCFFF3CFFCFFF3F3F3FFF00000FFFC0053
:1042F00000FFFFFFFCFFFFFFFFFFFFFFFFFFFFCF00
:10430000FFF3FFC00003FFC00003FFCFF3FFFFFF79
:10431000FCFFFFCFFCFFFFC000FFFFC003FFFFCF8C
:10432000FFFFFFFFFFFFFFFFFFFFFFFFFFFFFFCFCD
:10433000FFFFFFCFFCFFFFCFFCFFFFC000C3FFC0AC
:1043400000C3FFCFFFFFFFCFFFFFFFCFFFFFFFFF48
:10435000FFFFFFFFFFFFFFFFFFFFF3FFFCFFF3FF88
:10436000FCFFF3FFFCFFF3FFFCC3F00000C3FC0005
:1043700000FFFFFFFFFFFFFFFFFFFFFFFFFFFFFF4C
:10438000FFFFFFCFFFF3FFC00003FFC00003FFFFED
:104390000FFFFFCC00FFFFC0F0FFFFC3FCFFFFCF0C
:1043A000FCFFFFCFFFFFFFFFFFFFFFFFFFFFFFCF80
:1043B000FFFFFFCFFFF3FFCFFFF3FFC00003FFC0FE
:1043C0000003FFCFFFFFFFCFFFFFFFCFFFFFFFFF88
:1043D000FFFFFFFFFFFFFFFFFFFFFFCFFCFFFFC05F
:1043E00000FFFFC000FFFFFFFCFFFFC000FFFFC09A
:1043F00000FFFFFFFCFFFFC000FFFFC003FFFFCF78
:10440000FFFFFFFFFFFFFFCFFCFFFFC000FFFFC06C
:1044100000FFFFCFF3FFFFFFFCFFFFCFFCFFFFC05C
:1044200000FFFFC003FFFFCFFFFFFFFFFFFFFFFF06
:10443000FFFFFFFC0FFFFFF003FFFFC3F0FFFFCF05
:10444000FCFFFFCFFCFFFFCFFCFFFFC3F0FFFFF03F
:1044500003FFFFFC0FFFFFFFFFFFFFFFFFFFF3FF67
:10446000FCFFF00000FFF00000FFF3F3F3FFF3CFD9
:10447000FCFFFFCFFCFFFFC3F0FFFFF003FFFFFCDB
:104480000FFFFFFFFFFFFFFFFFFFFFFC0FFFFFF02E
:1044900003FFFFC3F0FFFFCFFCFFF3CFFCFFF3F3FD
:1044A000F3FFF00000FFF00000FFF3FFFCFFFFFF51
:1044B000FFFFFFFFFFFFFFCFFCFFFFCFFCFFFFC0B1
:1044C00000FFFFC000FFFFCFF3FFFFCFFCFFFFCFD8
:1044D000FCFFFFFFF0FFFFFFF3FFFFFFFFFFFFFF0A
:1044E000FFFFFFC3C3FFFFC300FFFFCF0CFFFFCFE2
:1044F0000CFFFFCC3CFFFFC030FFFFF0F0FFFFFFE1
:10450000FFFFFFFFFFFFFFFFFFFFFFFFFFFFFFFFBB
:10451000FCFFFFFFFCFFFFF00003FFC00003FFCF25
:10452000FCFFFFCFFCFFFFCFFCFFFFF3FFFFFFFF10
:10453000FFFFFFFFFFFFFFFFFFFFFFFFFCFFFFF09D
:1045400000FFFFC000FFFFCFFFFFFFCFFFFFFFF324
:10455000FCFFFFC000FFFFC000FFFFCFFFFFFFFF1A
:10456000FFFFFFFFFFFFFFFFFCFFFFFFC0FFFFFCA0
:1045700000FFFFC03CFFFFC3FFFFFFC03CFFFFFC8D
:1045800000FFFFFFC0FFFFFFFCFFFFFFFFFFFFFF7C
:10459000FCFFFFFF00FFFFC000FFFFC0FCFFFFF0BC
:1045A0003FFFFFFF0FFFFFF03FFFFFC0FCFFFFC01B
:1045B00000FFFFFF00FFFFFFFCFFFFFFFFFFFFCF3C
:1045C000FCFFFFCFFCFFFFC3F0FFFFC000FFFFFCBD
:1045D0000FFFFFC000FFFFC3F0FFFFCFFCFFFFCFC7
:1045E000FCFFFFFFFFFFFFFFFFFFFFFFFCFFF3FFED
:1045F000F0FFF3FF00FFF0F00CFFF003FFFFF3000C
:10460000FFFFFFF00CFFFFFF00FFFFFFF0FFFFFFCA
:10461000FCFFFFFFFFFFFFFFFFFFFFC3F0FFFFC037
:10462000FCFFFFCC3CFFFFCF3CFFFFCF0CFFFFCFD9
:10463000C0FFFFC3F0FFFFFFFFFFFFFFFFFFFFFF14
:10464000FFFFFFFFFFFFFFFFFFFFFFFF3FFFFF0039
:10465000000FFC00C003FCFFFFF3FFFFFFFFFFFFA5
:10466000FFFFFFFFFFFFFFFFFFFFFFFFFFFFFFFF5A
:10467000FFFFFFFFFFFFFFFFFFFFFFFFFFFFFC004C
:104680000003FC000003FFFFFFFFFFFFFFFFFFFF32
:10469000FFFFFFFFFFFFFFFFFFFFFFFFFFFFFFFF2A
:1046A000FFFFFFFFFFFFFCFFFFF3FC00C003FF0065
:1046B000000FFFFF3FFFFFFFFFFFFFFFFFFFFFFFB9
:1046C000FFFFFFFFFFFFFFFFFFFFFFFFCFFFFFFF2A
:1046D000F3FFFFFFF3FFFFFFCFFFFFFF3FFFFFFFF2
:1046E0003FFFFFFFCFFFFFFFFFFFFFFFFFFFFFFFCA
:1046F000FFFFFFFFFFFFFFFFFFFFFFFFFFFFFFFFCA
:10470000FFFFFFFFFFFFFFFFFFFFFFFFFCF003FFC7
:10471000FFFFFFFFFFFFFFFFFCF003FCF003FCF0D7
:1047200003FCF003FCF003FCF003FCF003FFFFFFCD
:10473000F0CCFFFF003FF0CCC3FF003FF0CCC3FF45
:10474000FFFFFFFFFFFF0C3FFF33CFF033C3FFC37B
:10475000CFFFFFFFFFFFFFFFFFFFFFF3CFFFF333AD
:10476000FF33CFFCCCFFFF3CFFFFFFFFFFFFFFFF4E
:104770000FFFFCF0FFFCCF3FFF3F3FFCCFFFFFFFF1
:10478000FFFFFFFFFFFFFFFFFFFFFFFCF3FFFFFF48
:10479000FFFFFFFFFFFFFFFFFFFFFFFFFFFFFFFC2C
:1047A000FF3FC3FFC3FFFFFFFFFFFFFFFFFFFFFF51
:1047B000FFC3FFC3FCFF3FFFFFFFFFFFFFFFFFFF44
:1047C000FFFFFFFFFFCFFFF0CFFFFF03FFF0CFFFA3
:1047D000FFCFFFFFFFFFF3FFFFF3FFFFF3FFFC003F
:1047E0000FFFF3FFFFF3FFFFF3FFFFFFFFFFFFFFED
:1047F000C3FFFFF03FFFFF3FFFFFFFFFFFFFFFFF94
:10480000FFFFFFF3FFFFF3FFFFF3FFFFF3FFFFF3F4
:10481000FFFFFFFFFFFFFFFFFFFFFC3FFFFC3FFF2E
:10482000FFFFFFFFFFFFFFFFFFFFFFFFF3FFFFFCA7
:104830003FFFFFC3FFFFFC3FFFFFC3FFFFFFFFFF83
:10484000FFFF000FFCFFF3FCFFF3FCFFF3FF000F83
:10485000FFFFFFFFFFFFFCFFFFFCFFF3FC0003FC7B
:10486000FFFFFCFFFFFFFFFFFFFFFFFC3FCFFCCF81
:10487000F3FCF3F3FCFCF3FC3F0FFFFFFFFFFFFF34
:10488000FF3FCFFCFFF3FCFCF3FCFCF3FF030FFF47
:10489000FFFFFFFFFFFFC3FFFFCCFFFFCF0FFCCFEA
:1048A000F3FC0003FCCFFFFFFFFFFF3FFFFCFC0317
:1048B000FCFCF3FCFCF3FF03F3FFFFFFFFFFFFFF34
:1048C000003FFCFCCFFCFCF3FCFCF3FF03F3FFFF19
:1048D000FFFFFFFFFFFFC3FFFFF3FC3FF3FFC0F34A
:1048E000FFFF03FFFFFFFFFFFFFF030FFCFCF3FCD5
:1048F000FCF3FCFCF3FF030FFFFFFFFFFFFFFCFCDB
:104900000FFCF3F3FCF3F3FF33F3FFC00FFFFFFFE4
:10491000FFFFFFFFFFFFFC3C3FFC3C3FFFFFFFFFB3
:10492000FFFFFFFFFFFFFFFFFFFFFFF0FFFFFC3C6C
:10493000CFFF3CCFFFFFFFFFFFFFFFF3FFFFCCFFE9
:10494000FFCCFFFF3F3FFCFFCFFCFFCFFFFFFFFF90
:10495000FFFFFFCCFFFFCCFFFFCCFFFFCCFFFFCC66
:10496000FFFFFFFFFCFFCFFCFFCFFF3F3FFFCCFF70
:10497000FFCCFFFFF3FFFFFFFFFFFFFFFFFFFFFC89
:10498000FF3FFCFFCFFFF3CFFFFC3FFFFFFFFFFF29
:10499000FFFC0003F3FFFCF3F0FCF3CF3CFCC0038F
:1049A000FFFFFFFCFFFFFC0FFFFCC033FFCFC3FC8A
:1049B000C03FFC0FFFFCFFFFFCFFF3FC0003FCFC0F
:1049C000F3FCFCF3FCFCF3FF030FFFFFFFFFFFFF13
:1049D000FF000FFCFFF3FCFFF3FCFFF3FF3FC3FFFF
:1049E000FFFFFCFFF3FC0003FCFFF3FCFFF3FF3FC2
:1049F000CFFFC03FFFFFFFFCFFF3FC0003FCFCF315
:104A0000FCF033FCFFF3FC3FC3FFFFFFFFFFFFFCA5
:104A1000FFF3FC0003FCFCF3FFF033FFFFF3FFFFA9
:104A2000C3FFFFFFFF000FFCFFF3FCF3F3FF03C323
:104A3000FFF3FFFFFFFFFCFFF3FC0003FCFCF3FFB1
:104A4000FCFFFCFCF3FC0003FCFFF3FFFFFFFCFF9B
:104A5000F3FCFFF3FC0003FCFFF3FCFFF3FFFFFF9D
:104A6000FFFFFFFF03FFFCFFF3FCFFF3FF0003FF6B
:104A7000FFF3FFFFFFFCFFF3FC0003FCF3F3FFF089
:104A8000FFFFCF33FC3FC3FCFFF3FFFFFFFCFFF34F
:104A9000FC0003FCFFF3FCFFFFFC0FFFFFFFFFFC2C
:104AA000FFF3FC0003FCFF03FFF0FFFCFF03FC002F
:104AB00003FCFFF3FCFFF3FC0003FCFF03FFC0FF5C
:104AC000FC3FF3FC0003FFFFF3FFFFFFFF000FFCC1
:104AD000FFF3FCFFF3FCFFF3FF000FFFFFFFFFFFFF
:104AE000FFFCFFF3FC0003FCF3F3FFF3F3FFFC0F09
:104AF000FFFFFFFFFFFFFF000FFCFFF3F0FFF3F0EE
:104B0000FFF3F3000FFFFFFFFCFFF3FC0003FCF3D8
:104B1000F3FFF3F3FFC3F3FF3C0FFCFFFFFFFFFFC7
:104B2000FC3F0FFF3CF3FCFCF3FCFCCFFF03C3FF97
:104B3000FFFFFFFFC3FFFFF3FCFFF3FC0003FCFFDD
:104B4000F3FFFFF3FFFFC3FFFFF3FF0003FCFFF3DF
:104B5000FCFFFFFCFFF3FF0003FFFFF3FFFFF3FF8A
:104B6000FF03FFC0F3FC3FFFFFC0F3FFFF03FFFFA6
:104B7000F3FFFFF3FF0003FCFFF3FF00FFFCFFF375
:104B8000FF0003FFFFF3FCFFF3FC3FC3FFCF3FFF3A
:104B9000F0FFFFCF3FFC3FC3FCFFF3FFFFF3FFFF3E
:104BA000C3FCFC33FC03FFFCFC33FFFFC3FFFFF33C
:104BB000FFFFFFFC3FC3FCCFF3FCF0F3FCFF33FC33
:104BC0003FC3FFFFFFFFFFFFFFFFFFC00003CFFF5B
:104BD000F3CFFFF3FFFFFFFFFFFFFFFFFFFFFFF339
:104BE000FFFC0FFFC3FFF03FFFFFFFFFFFFFFFFFD3
:104BF000FFFFFFFFFFCFFFF3CFFFF3C00003FFFF77
:104C0000FFFFFFFFFFFFFFFFFCFFFFFF3FFFFFC3B3
:104C1000FFFF3FFFFCFFFFFFFF3FFFFF3FFFFF3FA7
:104C2000FFFF3FFFFF3FFFFF3FFFFF3FFFFFFFFF94
:104C3000FFFFFFFFFFFFFFFFFFF3FFFFCFFFFFFFC0
:104C4000FFFFFFFFFFFFFF0CFFFCF33FFCF33FFC08
:104C5000F33FFC00FFFCFFFFFCFFF3FC0003FCFC48
:104C6000FFFCFF3FFCFF3FFF00FFFFFFFFFFFFFFD9
:104C7000FF00FFFCFF3FFCFF3FFCFF3FFF3C3FFF0F
:104C8000FFFFFFFFFFFF00FFFCFF3FFCFF3FFCFCBF
:104C9000F3FC0003FCFFFFFFFFFFFF00FFFCF33FFF
:104CA000FCF33FFCF33FFCF0FFFFFFFFFFFFFFFCC7
:104CB000FF3FFC000FFCFF33FCFF33FCFF33FFFF23
:104CC000FFFFFFFFFF00FFCCFF3FCCFF3FCCFCFF0F
:104CD000F0003FFFFF3FFCFFF3FC0003FCFCFFFF85
:104CE000FF3FFCFF3FFC00FFFCFFFFFFFFFFFCFF5F
:104CF0003FFCFF3FFC0033FCFFFFFCFFFFFFFFFF1B
:104D0000FFFFFFCFFF3FCFFF3FCFFF33F0003FFF5D
:104D1000FFFFFFFFFFFCFFF3FC0003FFF3FFFCC3FB
:104D20003FFC3C3FFCFF3FFFFFFFFFFFFFFCFFFF9F
:104D3000FCFFF3FC0003FCFFFFFCFFFFFFFFFFFC99
:104D4000FF3FFC003FFCFF3FFC00FFFCFF3FFC007F
:104D5000FFFCFFFFFCFF3FFC003FFCFCFFFFFF3FB1
:104D6000FCFF3FFC00FFFCFFFFFFFFFFFF00FFFC1D
:104D7000FF3FFCFF3FFCFF3FFF00FFFFFFFFCFFFB8
:104D80003FC0003FCCFCFFFCFF3FFCFF3FFF00FFAC
:104D9000FFFFFFFFFFFFFF00FFFCFF3FFCFF3FCCDB
:104DA000FCFFC0003FCFFF3FFFFFFFFCFF3FFC00C9
:104DB0003FFCFCFFFCFF3FFCFF3FFFFFFFFFFFFF4F
:104DC000FC3CFFFCF33FFCF33FFCF33FFF0C3FFFD9
:104DD000FFFFFFFFFFFFFF3FFF000FFCFF3FFCFF58
:104DE0003FFCFF3FFF3FFFFFFF3FFF003FFCFFFF98
:104DF000FCFFFFFF3F3FFC003FFCFFFFFFFF3FFFCB
:104E0000F03FFF0F3FFCFFFFFF0F3FFFF03FFFFFB3
:104E10003FFFFF3FFF003FFCFF3FFF03FFFCFF3F63
:104E2000FF003FFFFF3FFCFF3FFC3C3FFFC3FFFF96
:104E3000C3FFFC3C3FFCFF3FFFFFFFFFFF3FCFFCFA
:104E40003FCFC33FC03FFFCF0F3FFFF03FFFFF3FCC
:104E5000FFFFFFFC3C3FFCCF3FFCF33FFCFC3FFC73
:104E60003F3FFFFFFFFFFFFFFFFFFFFFCFFFF030E0
:104E70000FCFFFF3FFFFFFFFFFFFFFFFFFFFFFFF6E
:104E8000FFFFFFF00003FFFFFFFFFFFFFFFFFFFF3C
:104E9000FFFFFFFFFFCFFFF3F0300FFFCFFFFFFF5C
:104EA000FFFFFFFFFFFFFFFFCFFFFFF3FFFFCFFF7E
:104EB000FFCFFFFFF3FFFFFFFFFFFFFFFFFFFFFF3E
:104EC000FFFFFFFFFFFFFFF300FFFFFFFFFFFFFFFD
:104ED000F0FFFFFFF0FFFFCCCFF003CCCCF003FCE2
:104EE000CCFFFFF3CFC300FC33FFFFFFFFFF3FFF0B
:104EF00030F0CFFFCFFFFFF03FF303F0F3F3F3FF0A
:104F0000FFFFFFFFC0FFFFFFFFFFFFFFFFF003CF2B
:104F1000FCFFFFFFFFCFFCF003FFFFFFFFFFFFFFE2
:104F200033FFC0FF33FFFFFF3FFF3FF003FF3FFFB3
:104F30003FFFFFFFFFC3FFFCFFFFFFFFFFFF3FFF40
:104F40003FFF3FFFFFFFFFFFFFF3FFFFFFFFFFCF2D
:104F5000FFF0FFFF03FFFCFFFFFFFFFC03F3FCFC80
:104F600003FFFFF3FFF3FCF000F3FFF3FFFFFFF09D
:104F7000F3F33CF3C3FFFFFFFFF3F3F33CFCC3FF8A
:104F8000FFFFFFFF0FF333F000F33FFFFFFCC0F321
:104F9000CCFC3CFFFFFFFFFC03F3CCFC3CFFFFFF1E
:104FA000FFFFF0F03CFFC0FFFFFFFFFC33F3CCFC42
:104FB00033FFFFFFFFF3C3F33CFC03FFFFFFFFFFE3
:104FC000FFF3CFFFFFFFFFFFFFFFFFF3FFFCCFFF6C
:104FD000FFFF3FFF3FFCCFF3F3FFFFFFFFFF33FF78
:104FE00033FF33FFFFFFFFF3F3FCCFFF3FFF3FFF34
:104FF000FFFFF3F33CFFC3FFFFFFFFF003CFFCCF46
:105000003CCC03F0FFF30CFF30F30FF0FFF3FCF0A8
:1050100000F3CCF3CCFC33FFFFFC00F3FCF3F0FF18
:10502000FFF3FCF000F3FCF3FCFC03F3FCF000F3F3
:10503000CCF3FCF0F0F3FCF000F3CCFFFCFFF0FF4E
:10504000FFFC03F3FCF03CFF3FF3FCF000F3CCFF6C
:10505000CFF000FFFFF3FCF000F3FCFFFFFFFFFCCD
:105060003FF3FCFC00FFFCF3FCF000FF0FF030F31B
:10507000FCF3FCF000F3FCF3FFF0FFF000F3C0FFE3
:105080003FF3C0F000F3FCF000F3C3FC3CF000FF82
:10509000FFFC03F3FCF3FCFC03F3FCF000F33CFF28
:1050A0003CFFC3FFFFFC03F3FCF0FCF000F3FCF05B
:1050B00000F33CFF3CF0C3FFFFF3F0F3CCF030FF14
:1050C000FFFFF0F3FCF000F3FCFFF0FFFCFC00F34B
:1050D000FFF3FCFC00FFF0FC0CF3FFF03CFFC0FC16
:1050E00000F3FCFC0FF3FCFC00F3FCF0F0FF0FF00E
:1050F000F0F3FCFFF0F3CCF03FF3CCFFF0FFFFF058
:10510000F0F33CF3CCF0F0FFFFFFFFC000CFFCFF5B
:10511000FFFFFCFFC3F03FCFFFFFFFFFFFCFFCC04F
:1051200000FFFFFFFFFFFFFFCFFFF0FFCFFFFF3FBD
:10513000FF3FFF3FFF3FFFFFFFFFFFFFFFFFFCFFC2
:10514000F3FFFFFFFFF0FFF0CFF00FF3FFF3FCF0F2
:1051500000F3CFF3CFFC3FFFFFF00FF3CFF3CFFF10
:10516000FFFFFFFC3FF3CFF3CCF000FFFFFC0FF39A
:105170000FF30FFFFFFFFFF3CFF003F3CCFFFFFFB1
:10518000FFFC3F33CF33CFC00FF3FCF000F3CFFF72
:10519000CFF03FFFFFF3CFF00CF3FFFFFFFFFF3F28
:1051A000CF3FCC000FFFFFF3FCF000FF3FF00FF309
:1051B000CFFFFFF3FCF000F3FFFFFFF00FFFCFF096
:1051C0003FFFCFF03FF3CFF00FFFCFFFCFF03FFF18
:1051D000FFFC3FF3CFF3CFFC3F3FCF000F33CFF3C4
:1051E000CFFC3FFFFFFC3FF3CF333F000FFFFFF348
:1051F000CFF00FF3CFFFCFFFFFF3FFF30FFCCFFF95
:10520000FFFFCFFC03F3CFF3CFFCFFFFCFFC0FF387
:10521000FFF3CFF00FFFCFFF0FF0FFF0FFFF0FFC0A
:105220000FF3CFFC3FF3CFFC0FFFFFF3CFFC3FFCAE
:105230003FF3CFFFCF3C0F03FFFC0FFFCFFFFFF388
:10524000CFF0CFF30FF3CFFFFFFF3FF003CFFCFF13
:10525000FFFFFFFFFFC000FFFFFFFFFFFFCFFCF0DE
:1052600003FF3FFFFFFFFFFCFFFF3FFCFFFF3F820D
:10527000000000AA000000AAAA0000AAAAAA0055DD
:10528000AAAA0055555555AAAAAAAA55555555AAD0
:10529000AAAAAA15151515050505050101010100A4
:1052A00000000000000000000000000000000000FE
:1052B00000000000000000000000000000000041AD
:1052C00045F1FF5F5501000000000000EC520008AE
:1052D00000000020900400004A030008A0540008C9
:1052E00090040020B806000004010008C11BF8FF6C
:1052F000010A2E1F06213CFCFF013E320724FCFF61
:105300000F2580FFFF3F1AE01E291114FFFF03291C
:105310002A2A0F1139363A8F061B01FE06127F1A10
:10532000FC06120F1AF00612031DC01FF87F3F1B68
:105330001FF85611341EF8034318F8B31018490C1F
:105340002AF875111AF869297C292B294E39C619B2
:1053500083299C49064A0FD83A01846A1F063AF10C
:10536000063B01FC063A80062AF0069A81242906AB
:105370002AC0062A07423A7F482A0306197429C020
:10538000290629A91AF86A19064207021D782AFC7B
:105390004E433F040A2A20061A7C061BFCFF612BA1
:1053A00020FCF01A2010212A301E3A804E39542A4F
:1053B000F8064AF060390C59181144C03F3C2B38AC
:1053C000FCAD694819D6092C84493C29C049064AD4
:1053D00084CC290D19664906597E49064AE07E5A51
:1053E000FE8439423A3CBABB20FC0639DE11199ED4
:1053F0002906199612FCDA1C248A0C842A3E062AF5
:10540000F04E8A80EA3AC072198B1B3F040B1906D2
:105410002AFE069AE4AE49060930F03A7F06390CB6
:105420007A078A898449E4395A4A80604AC0664BBF
:10543000FC3F2A4BFC014849060A2B3F7E6984E960
:10544000C6093AD2A9540110400A030406080C10F8
:105450001820302D01020304043506070809948042
:10546000841E6917A93013A01C13080E1205139A85
:105470003613080B120413EE46130807120313B970
:105480004E130805920213391B1B08432C1AFB0804
:105490001AE5041315191B0835081A31041A2B0CC8
:0400000508000149A5
:00000001FF
